:100000000C941E060C9472280C949F280C9446069F
:100010000C9446060C9446060C9446060C94460630
:100020000C9446060C9446060C940E130C9446064B
:100030000C9446060C9446060C9446060C94460610
:100040000C94CC280C9446060C94BA2C0C94FD2CE1
:100050000C9446060C9446060C9446060C944606F0
:100060000C9446060C944606CA182C190B190E1946
:100070001119141917191A191D192C1926195E1A94
:10008000601A601A5E1A601A601A601A601A601AA2
:10009000601A601A601A601A601A601A601A601A90
:1000A000E419601A601A601A601A601A5519601A09
:1000B000601A601A601A601A601A601A601A601A70
:1000C000601A601A601A601A601A601AF019F01942
:1000D000F019F019F019F019F019F019F019601A67
:1000E000601A601A601A601A601A5519EF19EF1930
:1000F000EF19EF19601AFD19031A091A0F1A151AC8
:100100001B1A211A271A311A3B1A451A4F1A961927
:100110005819601A601A601A601AE419601A601A95
:10012000601A601A601A601A601A601AEE19EE19E5
:10013000EE19EE19601AFD19031A091A0F1A151A89
:100140001B1A211A271A311A3B1A451A4F1A9619E7
:100150005819601A601A601A601AE419931A931AEF
:10016000931A931A931A931A931A931A931A931A27
:10017000931A931A931AAA1BAA1BAA1BAA1BAA1B9F
:10018000AA1BD81AE21AEC1AF61A541B5E1B6D1B36
:100190007E1B061D1B1D271D301D3F1D641D6D1D73
:1001A000B61D7F1DC920CF20D520DC20EA200C21E0
:1001B0002A21456E746572206D656E752E2E2E0097
:1001C000546F67676C6564206D6963726F50504D42
:1001D00000546F67676C656420696E76657274653C
:1001E000642050504D2100546F67676C6564205443
:1001F00058206D7574696E672100546F67676C6570
:10020000642074656C656D65747279210050726F3D
:10021000746F636F6C206572726F72207769746897
:100220002052580054696D656F7574207768656E4B
:1002300020636F6E6E656374696E6720746F205201
:100240005800507265737320616E79206B65792058
:10025000746F2063616E63656C00436F6E6E6563DF
:1002600074696E6720746F2052582C20706F776508
:100270007220757020746865205258202877697440
:10028000682062696E6420706C7567206966206EF4
:100290006F74207573696E6720616C776179732064
:1002A00062696E642900546F67676C656420276912
:1002B0006D6D656469617465206F75747075742700
:1002C00000546F67676C65642027736C61766520E6
:1002D0006D6F64652700546F67676C6564202761E4
:1002E0006C776179732062696E642700546F676769
:1002F0006C65642050504D206368616E6E656C20A3
:100300006C696D69740053657420525353492069B8
:100310006E6A656374696F6E206368616E6E656C8A
:100320002028303D3D64697361626C652900536526
:10033000742050504D206D696E696D756D20737914
:100340006E630053657420626561636F6E20696E31
:1003500074657276616C0053657420626561636FC9
:100360006E2064656C617900536574206265616319
:100370006F6E206672657175656E637920696E2097
:10038000487A3A20303D64697361626C652C205074
:10039000783D504D52206368616E6E656C20782CFC
:1003A0002046783D465253206368616E6E656C202E
:1003B00078005365742050574D2073746F7020641B
:1003C000656C61792028302064697361626C6564B2
:1003D0002C20312D323535203D3D20302E317320FB
:1003E0002D2035306D696E29005365742050504DB5
:1003F0002073746F702064656C61792028302064EC
:10040000697361626C65642C20312D323535203D75
:100410003D20302E3173202D2035306D696E29003E
:10042000536574206661696C736166652064656CF0
:1004300061792028302064697361626C65642C20C6
:10044000312D323535203D3D20302E3173202D2089
:1004500035306D696E29002A2A2A2A2A2A2A2A2A50
:100460002A2A2A2A2A2A2A2A2A2A2A2A2A2A2A2AEC
:100470002A2A2A2A0052582041636B6564202D20C5
:1004800072657665727420737563636573736675E0
:100490006C21002A2A2A2A2A2A2A2A2A2A2A2A2AAD
:1004A0002A2A2A2A2A2A2A2A2A2A2A2A2A2A2A2AAC
:1004B000002A2A2A2A2A2A2A2A2A2A2A2A2A2A2AC6
:1004C0002A2A2A2A2A2A2A2A2A2A2A2A2A2A00528E
:1004D000582041636B6564202D20757064617465DC
:1004E000207375636365737366756C21002A2A2A0D
:1004F0002A2A2A2A2A2A2A2A2A2A2A2A2A2A2A2A5C
:100500002A2A2A2A2A2A2A2A2A2A0056616C696457
:100510002063686F69636573206172653A205B319F
:100520005D2D5B31365D20286368616E6E656C20E1
:10053000312D31362900536574206F7574707574D0
:1005400020666F7220706F727420005B585D2061AE
:10055000626F7274206368616E67657320616E6498
:10056000206578697420525820636F6E6669670051
:100570005B535D20736176652073657474696E6783
:100580007320746F205258005B525D20726576654F
:1005900072742052582073657474696E6773207486
:1005A0006F2064656661756C747300557365206EA9
:1005B000756D62657273205B312D445D20746F2010
:1005C0006564697420706F727473205B452D515D92
:1005D00020666F722073657474696E677300202DD6
:1005E00020726563656976657220636F6E66696700
:1005F000757261746F722C20727820737720000AF4
:100600000A6F70656E4C52536E67200053657420FC
:1006100073657269616C2062617564726174653AB8
:10062000200056616C69642063686F696365733A82
:100630002031202D20342B34202F2032202D203823
:10064000202F2033202D20382B34202F2034202D14
:10065000203132202F2035202D2031322B34202FF5
:100660002036202D20313600536574204368616E9A
:100670006E656C20636F6E6669673A20005365741F
:100680002044617461726174652028302D32293AEA
:10069000200053657420486F70206368616E6E653A
:1006A0006C7320286D61782032342C207365706162
:1006B000726174656420627920636F6D6D61732966
:1006C0002076616C69642076616C75657320312DCC
:1006D0003235353A2000536574206368616E6E656B
:1006E0006C2073706163696E6720287831306B48C5
:1006F0007A293A200053657420524620706F77653E
:10070000722028302D37293A200053657420524634
:10071000206D6167696320286865782920652E67E8
:100720002E20307844454144463030443A2000532E
:1007300065742062617365206672657175656E63AC
:10074000792028696E20487A293A20005B5A5D207A
:10075000656E746572207265636569766572206383
:100760006F6E66696775726174696F6E2075746902
:100770006C79005B465D20646973706C61792061FF
:10078000637475616C206672657175656E63696509
:10079000732075736564005B525D2063616C6375E3
:1007A0006C6174652072616E646F6D206B65792079
:1007B000616E6420686F70206C697374005B495DC2
:1007C000207265696E697469616C697A6520736508
:1007D0007474696E677320746F20736B65746368DB
:1007E0002064656661756C7473005B585D2072658A
:1007F00076657274206368616E67657320616E64EC
:100800002065786974206D656E75005B535D20739B
:100810006176652073657474696E677320746F20E8
:10082000454550524F4D20616E64206578697420B3
:100830006D656E7500557365206E756D62657273BA
:10084000205B302D395D20746F20656469742070E1
:100850006172616D657465727300202D2053797328
:1008600074656D20636F6E66696775726174696F18
:100870006E000A0A6F70656E4C52536E672000510D
:1008800029204F7574707574206265666F726520DB
:100890006C696E6B20283D465329203A2000502970
:1008A00020536C617665206D6F64652028657870D3
:1008B0006572696D656E74616C293A20004F29205C
:1008C00054696D65642042494E44206174207374FC
:1008D000617274757020203A20004E292050504DCE
:1008E000206F7574707574206C696D69746564200F
:1008F000202020203A200044495341424C454400E6
:100900004D292050504D205253534920746F20637D
:1009100068616E6E656C202020203A20004C2920F2
:1009200050504D206D696E696D756D2073796E63E1
:10093000202875732920203A200044495341424C15
:100940004544004B29204661696C736166652062ED
:100950006561636F6E20696E74762E2028312D32AA
:10096000353573293A20004A29204661696C736144
:10097000666520626561636F6E2064656C617920D5
:1009800028302D323535203D3E20313073202D204A
:100990003135306D696E293A200049292046616958
:1009A0006C7361666520626561636F6E206672714B
:1009B0002E203A200048292050574D2073746F7024
:1009C0002064656C6179202020202020203A2000BE
:1009D00047292050504D2073746F702064656C61FE
:1009E00079202020202020203A200046292046611E
:1009F000696C736166652064656C617920202020D4
:100A00002020203A200050574D206368616E6E65AB
:100A10006C200066756E6374696F6E3A2000292041
:100A2000706F72742000506F776572546F776572C3
:100A300000445446205548462033322D62697420C4
:100A400031306368004F70656E4C52536E67525878
:100A5000206D696E6920342F36636800466C7974A6
:100A6000726F6E2F4F72616E6765525820554846FF
:100A70002038636800525820747970653A20004429
:100A8000697361626C656400487A00203D3D200016
:100A900043616C63756C61746564207061636B6540
:100AA0007420696E74657276616C3A200042292068
:100AB0004D6963726F202868616C66292050504D23
:100AC000202020203A00412920496E766572746505
:100AD000642050504D20696E20202020203A0030A4
:100AE00029204D7574652062757A7A657220286DAB
:100AF0006F73746C79293A003929205365726961E2
:100B00006C2062617564726174653A00736D617224
:100B100074506F7274004672536B79005472616E38
:100B200073706172656E740044697361626C6564B0
:100B30000038292054656C656D657472793A2020FF
:100B40002020202020003729204368616E6E656CCC
:100B500020636F6E6669673A202000362920446161
:100B60007461726174652028302D32293A2020206A
:100B700000352920486F70206368616E6E656C7364
:100B80003A2020202020003429204368616E6E65C1
:100B90006C2073706163696E673A202000332920EE
:100BA000524620706F7765722028302D37293A2001
:100BB0002020003229205246206D616769633A2067
:100BC0002020202020202020003129204261736530
:100BD000206672657175656E63793A202020000089
:100BE00000000700020100000304060000000000EE
:100BF00000000001020408102040800102040810D7
:100C00002001020408102004040404040404040263
:100C10000202020202030303030303000000002395
:100C2000002600290000000000250028002B0000FD
:100C3000000000240027002A0000EB2D11241FBE15
:100C4000CFEFD8E0DEBFCDBF13E0A0E0B1E0E4EE2F
:100C5000F1E602C005900D92A83CB107D9F716E065
:100C6000A8ECB3E001C01D92AE38B107E1F71CE07B
:100C7000CCE3DCE004C02297FE010E94F42ECA33CC
:100C8000D107C9F70E94272E0C94F0300C94000075
:100C900080917305813019F482E08093730580910F
:100CA0007305833019F484E0809373050895A89543
:100CB0000895DC01ED91FC910190F081E02D099502
:100CC00008952091740530917505382748E0C901D1
:100CD000880F991F37FF06C09C0151E2252750E17C
:100CE000352701C09C01415091F730937505209341
:100CF0007405089588E38093760580E092ECA1E086
:100D0000B0E08093770590937805A0937905B09330
:100D10007A0587E08093830580EC9AECA9E8B6E336
:100D200080937B0590937C05A0937D05B0937E0511
:100D300085E0809384058DEE9EEFADEABEED809355
:100D40007F0590938005A0938105B0938205E5E827
:100D5000F5E080E090E0863028F4DC01AE54BC4F32
:100D60002C9101C020E0219301968831910599F7DB
:100D700082E080939D058AE080939E05089580EC33
:100D800097EFAAEBB7E38093BB059093BC05A093C4
:100D9000BD05B093BE0580E090E0A0E0B0E5809393
:100DA000BF059093C005A093C105B093C205E3ECC5
:100DB000F5E080E081938F5F8031E1F70895A0E056
:100DC000B0E0E5EEF6E00C94BD2ED82F0E9422296B
:100DD0006115710581059105C9F30E94602F10927C
:100DE0007F05109280051092810510928205C4E063
:100DF000812C912C54018A94C0907F05D09080055D
:100E0000E0908105F0908205FE2CED2CDC2CCC24AA
:100E10000E945B2FA50194010E949C2E6C0D7D1DEC
:100E20008E1D9F1D60937F057093800580938105C3
:100E300090938205C15001F7DD2309F450C005E805
:100E400015E0E801A12CB12C62E3C62ED12CE12CD7
:100E5000F12C8881882309F442C0B39419F40E94CC
:100E60007A063DC00E945B2FA70196010E949C2E2E
:100E7000E1E0E60FA5E8B5E08A2F801B8A1520F493
:100E80008D918E13F9CFE9CF2091840530E0A0E158
:100E9000B7E20E94342E9B01AC01AE2FB0E00E945D
:100EA000432E40907B0550907C0560907D057090AE
:100EB0007E05640D751D861D971D4090BB055090E5
:100EC000BC056090BD057090BE05461657066806C5
:100ED000790618F2E993A39488E1A812BACFCDB7A6
:100EE000DEB7E0E10C94D92E8436910520F4BC01E4
:100EF00080E090E017C09C018E3B910528F42A55B4
:100F00003109AAE0B0E00CC0823D910528F4245BD1
:100F10003109A4E6B0E004C02D5C3109A8E5B2E0D7
:100F20000E94342EA4E6B0E09B01AC010E94432E47
:100F3000089590E08C599F4F0E947407089582E0B5
:100F40008093B00085E08093B10061E083E00E946F
:100F5000CF2960E083E00E94082A08950097C9F035
:100F60009C0140E050E068E478EE81E090E00E946F
:100F70009C2E2F3F31054105510529F020F02FEF20
:100F800030E040E050E02093B3008091B0008061F9
:100F900003C08091B0008F7E8093B000089560E020
:100FA0008CE00E94CF2961E08BE00E94CF2961E0B4
:100FB0008DE00E94CF2960E082E00E94CF2961E0AD
:100FC00084E00E94CF29089542E050E068E476E092
:100FD00080E00E9452280895E3E0F0E089E08093E9
:100FE0005700E491E67081E0E63009F080E0089572
:100FF000CF93DF93C82F0E94EC07882381F0DFB7DF
:1010000081E080937205F8940E94570688E18093EE
:101010006000C0936000C1110E945706DFBFDF91DE
:10102000CF9108958F929F92AF92BF92CF92DF920D
:10103000EF92FF92CF93FC01C0A5EC2FE770F0E098
:10104000E658FC4FA081B0E0C7FF03C024E130E0C8
:1010500002C02FE030E0FC0197A183E1989FF001EE
:101060001124E25CFE4F80809180A280B380A20FA9
:10107000B31F20E43FE14DE750E00E944E2EA50152
:1010800094010E947A2E8C2F887149F469017A01AB
:10109000E0EDCE0EE7E0DE1EE11CF11C1BC0C7FF39
:1010A00005C060E47AE88CE29EE004C060E07EEE79
:1010B0008AEB9BE069017A01F8EBCF0EFBE0DF1EC3
:1010C000E11CF11CA50194010E947A2EC20ED31ED0
:1010D000E41EF51EC701B60169517C4F8F4F9F4F2B
:1010E00028EE33E040E050E00E947A2EA8EEB3E014
:1010F0000E94432ECF91FF90EF90DF90CF90BF9052
:10110000AF909F908F9008958F3F910551F048F0D8
:10111000811522E0920738F08115934030F482E087
:10112000089580E0089581E0089583E00895A0E0A7
:10113000B0E0EDE9F8E00C94C62EEB018A01B82F7F
:10114000B695A0E028813981F80120832A813B816E
:1011500021832C813D8122832E813F8123836881DD
:1011600079814A815B812C813D81EE81FF819F2FB6
:101170009295990F990F907C272F2370922B252FF2
:101180002370220F220F922B232F23702295207F72
:10119000922BF80194830B5F1F4F2896AF5FBA170D
:1011A00088F680FF24C0888199810E948408D82E07
:1011B0008A819B810E948408E82E8C819D810E94F7
:1011C0008408F82E8E819F810E948408F0E4DF9EBF
:1011D000A001112490E1E99E90011124242B282BD9
:1011E000E4E0FE9EB0011124262BF8012083CDB748
:1011F000DEB7E7E00C94E22E803223E0920708F19C
:10120000883E23E0920740F48F519340E4E09695A6
:101210008795EA95E1F70895803D27E0920718F455
:101220008C5D93400895883928E0920768F4885CC3
:10123000974074E0969587957A95E1F78D509C4F8D
:10124000089580E090E008958FEF93E008958C304A
:10125000910540F4A4E0880F991FAA95E1F7885DF5
:101260009C4F0895843F23E0920718F484529C4FCA
:101270000895811524E0920740F48657934FF4E0D7
:10128000880F991FFA95E1F7089580E998E008958D
:101290009C013695279525753575821B930B9C010E
:1012A0002373337396958795969587958373937378
:1012B000820F931F9C0154E0369527955A95E1F7CC
:1012C000280F391F2F703F7041E051E0249FC0016B
:1012D000259F900D349F900D1124892F08952D98EE
:1012E000882319F000002B9A02C000002B98000000
:1012F0002D9A000008952D9A000083B12D980000CA
:10130000829581700895CF93DF93D82F5C9A2D98A2
:101310005C98C8E08D2F80780E946F09DD0FC15066
:10132000C9F72D98DF91CF9108958F770E94830997
:101330000895CF93DF93D82FC8E08D2F80780E9437
:101340006F09DD0FC150C9F72D98DF91CF91089536
:10135000CF93DF932D98C8E080E0D82FDD0F0E9457
:101360007B098D0FC150C9F7DF91CF9108950E947D
:1013700095090E94A8095C9A0895A1E0B0E0E3EC09
:10138000F9E00C94CB2E806869830E9483096981FF
:10139000862F0E9499095C9A2196E2E00C94E72E30
:1013A000CF93C0917F05C827E82FF0E0EA58FA4FA5
:1013B000678589E70E94BD096C2F8DE30E94BD09F6
:1013C0006C2F82E40E94BD09CF91089586E20E94AD
:1013D000B7090895CF93DF93EC016C818CE10E94F3
:1013E000BD096D818DE10E94BD096E818EE10E9473
:1013F000BD096F8180E20E94BD09688581E20E947B
:10140000BD09698582E20E94BD096A8583E20E9466
:10141000BD096B8584E20E94BD096C8585E20E944E
:10142000BD096D858AE20E94BD096E858EE60E9427
:10143000BD096F858FE60E94BD09688980E70E941B
:10144000BD09698981E70E94BD096A8982E70E9416
:10145000BD09DF91CF910895CF92DF92EF92FF9275
:10146000CF93DF936B017C01C11488E3D8068CE92C
:10147000E8068CE1F80628F5C701B60120E836E950
:1014800048E950E00E947A2EE901689760E879E621
:1014900087E69FEF0E94562E6C0D7D1D8E1D9F1DB1
:1014A000F2E0660F771F881F991FFA95D1F721E7A1
:1014B00032E040E050E00E947A2EF22EE32E80E4EB
:1014C00021C0C701B60120E03DE241E351E00E94A6
:1014D0007A2EE901689760E073ED8EEC9EEF0E9432
:1014E000562E6C0D7D1D8E1D9F1D660F771F881F4C
:1014F000991F21E732E040E050E00E947A2EF22E60
:10150000E32E80E66C2F6F71680F85E70E94BD099E
:101510006E2D86E70E94BD096F2D87E70E94BD09E9
:10152000DF91CF91FF90EF90DF90CF900895682FDB
:101530008DE60E94BD0908958F929F92AF92BF924F
:10154000CF92DF92EF92FF92CF93DF93D82F61E09B
:1015500089E00E94082A62E370E080E090E00E9447
:10156000452960E089E00E94082A62E370E080E09B
:1015700090E00E94452983E00E94B709809371059D
:1015800084E00E94B7098093700560E086E00E94C5
:10159000BD0961E087E00E94BD096FE789E00E9414
:1015A000BD0965E08AE00E94BD0965E18BE00E940B
:1015B000BD0962E18CE00E94BD096DEF8DE00E94E3
:1015C000BD0960E08EE00E94BD09DD2319F08BE2C9
:1015D00091E008C020919D0533E1239FC0011124B3
:1015E000825C9E4F0E94EA096CE880E30E94BD097C
:1015F0006FE082E30E94BD0962E483E30E94BD09BB
:1016000080919E0587FF02C064E101C06AE084E327
:101610000E94BD096AE285E30E94BD096DE286E38E
:101620000E94BD0964ED87E30E94BD0960E088E384
:101630000E94BD0960E089E30E94BD09D11109C083
:10164000C0907F05D0908005E0908105F0908205E4
:1016500007C0C5E9CC2EC1ECDC2EED2CCEEDFC2E66
:10166000CAE38F2C9924AA24BB24682D8C2F0E94B6
:10167000BD09682D85E08C0F0E94BD09FE2CED2C64
:10168000DC2CCC24CF5FCE3361F76FEF83E40E9474
:10169000BD096FEF84E40E94BD096FEF85E40E94ED
:1016A000BD096FEF86E40E94BD09DD2311F066E0FD
:1016B00002C0609183058DE60E94BD0960E089E764
:1016C0000E94BD09609184058AE70E94BD0960E01F
:1016D00083E70E94BD0960E084E70E94BD09D11143
:1016E00009C060917B0570917C0580917D0590918A
:1016F0007E0504C060EC7AEC89E896E30E942C0A2F
:10170000DF91CF91FF90EF90DF90CF90BF90AF909F
:101710009F908F90089561E087E00E94BD0964E288
:101720008EE70E94BD0963E088E00E94BD0960E089
:1017300088E00E94BD0965E087E00E94BD0962E083
:1017400085E00E94BD0983E00E94B709809371057E
:1017500084E00E94B70980937005089583E00E9499
:10176000B7098093710584E00E94B70980937005E2
:1017700061E087E00E94BD096AE070E080E090E0EF
:101780000E9445290E948B0B00000895CF92DF92A2
:10179000FF920F931F93CF93DF931F92CDB7DEB7C6
:1017A000082F162F8EE399830E94BD09F02EC02EBC
:1017B0009981D92E8C2D8F19811738F4F6016191FA
:1017C0006F018FE70E94BD09F5CF64E085E00E94BC
:1017D000BD0983E00E94B7098093710584E00E94EF
:1017E000B709809370050E94222960936C0570935D
:1017F0006D0580936E0590936F0569E087E00E9408
:10180000BD0981E0809373050F90DF91CF911F9107
:101810000F91FF90DF90CF9008950F931F930E9438
:10182000C60B80917305813099F40E9422290091A2
:101830006C0510916D0520916E0530916F05601B50
:10184000710B820B930B603A76488140910548F307
:1018500080917305813031F46EE971E082EE95E09C
:101860000E940E2B1F910F9108950F931F9380914B
:101870007305823021F41092730581E020C08091BD
:1018800073058130D9F40E94222900916C051091D2
:101890006D0520916E0530916F05601B710B820BF9
:1018A000930B613A76488140910540F061E087E012
:1018B0000E94BD091092730582E001C080E01F9173
:1018C0000F910895CF93DF93EC014AE050E06D2F24
:1018D00070E082EE95E00E94DC2B6EE282EE95E0F5
:1018E0000E94E02ABE0184E0769567958A95E1F72B
:1018F0006F7077274AE050E082EE95E00E94DC2B83
:10190000DF91CF910895D82FC0E0CD1780F45E9A73
:1019100064E670E080E090E00E9445295E9864E60D
:1019200070E080E090E00E944529CF5FEECF6CE24E
:1019300071E080E090E00E944529E6CF0F931F936D
:10194000CF93DF93EC01062F15E0115051F0CE013B
:101950000E94D730081741F0602FCE010E94DF307F
:10196000F4CF82E00E94830CDF91CF911F910F9101
:101970000895A0E0B0E0EFEBFCE00C94BD2E482E03
:10198000562EC0E0D0E0612C712CE12CF12C00E04F
:1019900010E041100CC06090D40586E4689E3001D0
:1019A000112459E1E52EF12C0AEB15E01EC091E05F
:1019B00049120FC06090D405E6E46E9E30011124F8
:1019C000FBE16F0E711C49E2E42EF12C06E715E0F5
:1019D0000CC082E0481209C028E1622E772473947B
:1019E000EE24E394F12C03ED15E043018C0E9D1ED3
:1019F00010927505109274053401A62CA818B12C0C
:101A0000C30101966C01AE14BF04A8F4A00EB11E70
:101A1000511006C0C3010E94D730F501808305C074
:101A2000F5016081C3010E949E0CF50180810E9436
:101A300061063601E2CFC301511018C0C3010E94F4
:101A4000D730B82EC6010E94D7302B2D30E0322F70
:101A50002227282B80917405909175058217930792
:101A600079F4C0E0D0E05524539493CF36016091CF
:101A700075050E949E0C60917405C6010E949E0C23
:101A8000C05EDE4FC13E92E0D90708F482CF852DBB
:101A9000CDB7DEB7E0E10C94D92E61E082E00E9480
:101AA000B90C089560E082E00E94B90C8091D305E2
:101AB000853028F084E08093D3050E944D0D8091FD
:101AC000D3058093D405089561E080E00E94B90CAD
:101AD00061E081E00E94B90C089560E080E00E941E
:101AE000B90C882351F060E081E00E94B90C882392
:101AF00021F080917605883349F00E94BF060E944C
:101B00007A0681E00E94DF060E94640D0895882312
:101B100019F06AEA71E002C06EEA71E082EE95E0C7
:101B20000E940E2B0895FF920F931F93CF93DF9384
:101B300069EC7BE082EE95E00E94BA2A40917B0539
:101B400050917C0560917D0570917E052AE030E022
:101B500082EE95E00E94E32B63EB7BE082EE95E062
:101B60000E94BA2A40917F055091800560918105BD
:101B70007091820520E130E082EE95E00E94E32B37
:101B80006DE97BE082EE95E00E94BA2A4AE050E0DF
:101B90006091830582EE95E00E940B2C67E87BE064
:101BA00082EE95E00E94BA2A4AE050E060918405F6
:101BB00082EE95E00E940B2C61E77BE082EE95E0DF
:101BC0000E94BA2AC5E8D5E0F12C8E0188818823CD
:101BD000A9F0FF2031F061EB71E082EE95E00E9408
:101BE000DD2A21964AE050E0F801608182EE95E01E
:101BF0000E94D42BF394F8E1FF12E7CF82EE95E038
:101C00000E94E82A6BE57BE082EE95E00E94BA2A0A
:101C10004AE050E060919D0582EE95E00E940B2C19
:101C200066E47BE082EE95E00E94BA2AE0919E0590
:101C3000E770F0E0EE0FFF1FEE57FC4F60817181FF
:101C400082EE95E00E940E2B61E37BE082EE95E050
:101C50000E94BA2A80919E058871883069F028F424
:101C6000811113C068E27BE00CC0803141F0883103
:101C700061F46CE07BE005C06CE17BE002C066E1F2
:101C80007BE082EE95E00E94FC2A68EF7AE082EE2B
:101C900095E00E94BA2A40917705509178056091AD
:101CA000790570917A052AE030E082EE95E00E9495
:101CB000E32B6FED7AE082EE95E00E94BA2A8091E4
:101CC000BF0580710E94870D66EC7AE082EE95E098
:101CD0000E94BA2A8091BF0580740E94870D6DEA28
:101CE0007AE082EE95E00E94BA2A8091BF05807268
:101CF0000E94870D60E97AE082EE95E00E94BA2AA0
:101D000086E795E00E941208AB01BC012AE030E0B2
:101D100082EE95E00E94C52B6BE87AE082EE95E0BA
:101D20000E94BA2A86E795E00E9412089B01AC0146
:101D300060E472E48FE090E00E947A2EBA01A9017B
:101D40002AE030E082EE95E00E94C52B68E87AE058
:101D500082EE95E00E94FC2ACDB7DEB7E5E00C9458
:101D6000E42E8F929F92AF92BF92CF92DF92EF922A
:101D7000FF92811107C06FE77AE082EE95E00E9442
:101D8000FC2A2FC090E00E94740724E630E040E077
:101D900050E00E947A2ECA01B9012AE030E040E00A
:101DA00050E00E947A2E49015A016B017C012AE021
:101DB00030E0B501A40182EE95E00E94C52B6EE2F1
:101DC00082EE95E00E94E02A2AE030E0B701A60109
:101DD00082EE95E00E94C52B63E782EE95E00E94BB
:101DE000202BFF90EF90DF90CF90BF90AF909F900F
:101DF0008F9008951F93CF93DF9365E77AE082EE8B
:101E000095E00E94BA2A80919F05813041F46CE5EB
:101E10007AE082EE95E00E94FC2A10E050C0823009
:101E200019F465E47AE0F5CF843019F461E37AE0DF
:101E3000F0CF853091F766E27AE0EBCFC12FD0E0AA
:101E4000C930D1050CF441C068E3610F82EE95E022
:101E50000E94E02A6EE17AE082EE95E00E94BA2AC2
:101E6000BE016F5F7F4F4AE050E082EE95E00E9436
:101E7000A42B63E17AE082EE95E00E94BA2AC15673
:101E8000DA4FE981E03218F566E07AE082EE95E01B
:101E90000E94BA2A8981803130F06DE673E082EECB
:101EA00095E00E94DD2A69816F7070E06F5F7F4F5F
:101EB0004AE050E082EE95E00E94AD2B1F5F8091DA
:101EC0004805181708F4BACF0FC061E3BECFEF7012
:101ED000F0E0EE0FFF1FEE56FC4F6081718182EE45
:101EE00095E00E940E2BEACF6BEE79E082EE95E052
:101EF0000E94BA2A8091B7050E94B10E60ED79E088
:101F000082EE95E00E94BA2A8091B8050E94B10E37
:101F100065EB79E082EE95E00E94BA2A8091B905DE
:101F20000E94B10E6AE979E082EE95E00E94BA2A39
:101F30004091AF055091B0056091B1057091B20527
:101F4000411551056105710539F12AE030E082EE55
:101F500095E00E94E32B67E679E082EE95E00E942F
:101F6000BA2A8091B3050E949907AB01BC012AE00F
:101F700030E082EE95E00E94E32B63E479E082EEAC
:101F800095E00E94BA2A4AE050E06091B40582EEE2
:101F900095E00E940B2C06C06AE379E082EE95E0A2
:101FA0000E94FC2A6DE179E082EE95E00E94BA2A57
:101FB0006091B5057091B6054AE050E082EE95E07B
:101FC0000E94F52B60E079E082EE95E00E94BA2A4B
:101FD0006091AE05603450F470E06F5F7F4F4AE06F
:101FE00050E082EE95E00E94AD2B06C067EF78E0EE
:101FF00082EE95E00E94FC2A6AED78E082EE95E0A0
:102000000E94BA2A8091AD0580FF03C063EB71E0A6
:1020100002C067EB71E082EE95E00E940E2B6DEB43
:1020200078E082EE95E00E94BA2A8091AD05827038
:102030000E94870D6EE978E082EE95E00E94BA2A50
:102040008091AD0584700E94870D6FE778E082EE85
:1020500095E00E94BA2A8091AD0588700E94870D94
:10206000DF91CF911F9108950F931F93CF93DF932B
:10207000209145052F3FA9F56FEF75E082EE95E0C1
:102080000E94BA2A80E893E00E94620C6EED75E02F
:1020900082EE95E00E94BA2A80914605909147050C
:1020A0000E94620C6BEA75E082EE95E00E94FC2AC9
:1020B00068E875E082EE95E00E94FC2A60E775E032
:1020C00082EE95E00E94FC2A6BE475E082EE95E0DA
:1020D0000E94FC2A82EE95E00E94E82A0E94FA0EF5
:1020E00068C012160CF065C0332727FD309580912B
:1020F000480590E0821793070CF45BC066E375E037
:1021000082EE95E00E94BA2A60914505772767FD27
:1021100070954AE050E082EE95E00E94AD2B6BE0B6
:1021200075E082EE95E00E94BA2A10E008E2809104
:1021300049051817D0F5C12FD0E0CC0FDD1FC65BC5
:10214000DA4F288130E080914505992787FD9095E9
:1021500001972817390739F56BEB71E082EE95E0AE
:102160000E94DD2A4AE050E0602F82EE95E00E9456
:10217000D42B6FEB71E082EE95E00E94DD2AE981BD
:10218000EF70F0E0EE0FFF1FEE56FC4F60817181A3
:1021900082EE95E00E94DD2A63EC71E082EE95E02C
:1021A0000E94DD2A0F5F1F5FC2CF82EE95E00E9482
:1021B000E82ADF91CF911F910F910895FF920F931D
:1021C0001F93CF93DF93C5E8D5E0F12C8E01888172
:1021D0008823D1F165EC71E082EE95E00E94DD2A62
:1021E0004AE050E06F2D82EE95E00E94D42B62ED24
:1021F00071E082EE95E00E94DD2A2196F8012081AF
:1022000030E0A0E1B7E20E94342E9B01AC01A09126
:102210008405B0E00E94432EAB01BC0180917B0598
:1022200090917C05A0917D05B0917E05480F591FC6
:102230006A1F7B1F2AE030E082EE95E00E94E32BCC
:10224000F394F8E1FF12C2CFCDB7DEB7E5E00C940E
:10225000E42E1092DF0485E6E0EEF4E0DF011D924B
:102260008A95E9F70895CF93C82F8F3719F08830F2
:1022700009F045C0E091DF04EE23D9F1E150E0938D
:10228000DF04F0E0E052FB4F10826DE070E082EE80
:1022900095E00E945906C0E08091DF04C81760F401
:1022A000EC2FF0E0E052FB4F608170E082EE95E0B1
:1022B0000E945906CF5FF0CF60E270E082EE95E0B9
:1022C0000E9459066DE070E082EE95E00E9459068A
:1022D000C0E08091DF04C81778F5EC2FF0E0E05201
:1022E000FB4F608170E082EE95E00E945906CF5F5F
:1022F000F0CF67E082EE95E00E94E02A1DC08B31AE
:1023000019F40E9429111AC08D30C1F08A30B1F041
:102310008091DF04843668F76C2F70E082EE95E0E0
:102320000E945906E091DF0481E08E0F8093DF0464
:10233000F0E0E052FB4FC08380E001C081E0CF912C
:102340000895CF93C82F0E9422296093C8047093E8
:10235000C9048093CA049093CB04C093DD04CC23BA
:1023600029F040E051EE60E070E004C040E855E242
:1023700060E070E082EE95E00E946A2DCF910895B2
:102380009091CC04492F4F7050E0BA016F5F7F4F9E
:10239000292F30E0E4E035952795EA95E1F76217BB
:1023A000730759F0FA01E353FB4F808381E0890FF3
:1023B0008F70907F892B8093CC0408956EE770E036
:1023C00082EE95E00E9459060895A3E1B1E0EBEE9C
:1023D000F1E10C94BE2EE5E8F5E0712C81918823A3
:1023E00021F0739428E17212F9CF66ED71E082EE6C
:1023F00095E00E940E2B4AE050E0672D82EE95E0BA
:102400000E940B2C80E00E949C0A0E948B0B8E0184
:102410000E5F1F4FC12CD12C7601C39466246A94A1
:102420005C2C0E9416294B015C012091840530E050
:10243000A0E1B7E20E94342E9B01AC01C701B601B6
:102440000E94562E20917B0530917C0540917D05A0
:1024500050917E05620F731F841F951F2091BB054D
:102460003091BC054091BD055091BE052617370738
:102470004807590718F4F801608225C08C2D0E9486
:10248000D00961E070E080E090E00E944529F80109
:1024900010820E941629681979098A099B09643FEC
:1024A00071408105910540F40E94E609F801908190
:1024B000981778F78083EDCF50FE03C05D985E9A41
:1024C00002C05D9A5E982FEFC21AD20AE20AF20A9F
:1024D0000F5F1F4F8FEFC816D104E104F10409F01C
:1024E0009FCFCE019395FC01D82E7FEF68EC2E2F65
:1024F000281B271510F051E056C0DE01129651E05E
:102500002FEF41E03D91321710F0322F01C0452FDF
:102510005F5F5F3F11F0232FF5CF4193242F30E011
:10252000A1E0B0E0AC0FBD1FA20FB31F5C93413020
:1025300079F0DE01A20FB31F5C93423049F0AFEF98
:10254000BFEFAC0FBD1FA20FB31F6C934E3F78F6C9
:10255000A2E0B0E0AC0FBD1FA20FB31F7C934D3FB4
:1025600030F6A3E0B0E0AC0FBD1FA20FB31F6C9319
:10257000BECF452F242F30E0FC01E20FF31F608116
:10258000AFEFB0E0AC0FBD1FA20FB31F2C916217CD
:1025900048F44150DC01A40FB11D2C9120836C93B1
:1025A0004111E8CF5F5F571520F3372D369520E0B6
:1025B000231770F4DC01A20FB11D4C91522F530F61
:1025C000FC01E50FF11D50815C9340832E5FF0CF3D
:1025D000F5E8EF2EF5E0FF2E8C01802F8D19871581
:1025E00098F4F801C1908F014AE050E06C2D82EE22
:1025F00095E00E94D42B6CE282EE95E00E94E02AE6
:10260000F701C1927F01E9CF82EE95E00E94E82AAE
:1026100081E0CD5EDE4FEFE00C94DA2E1F920F9238
:102620000FB60F9211241F932F933F934F935F93F5
:102630006F937F938F939F93AF93BF93CF93DF93CA
:10264000EF93FF93C0918600D0918700809187041B
:10265000909188042091A904211155C09E01281B46
:10266000390B8091BF059091C005A091C105B09133
:10267000C20585FD02C036952795253C49E0340703
:10268000B8F140910A0150E060E070E02CE1B695AD
:10269000A795979587952A95D1F70097A105B1053C
:1026A00021F481E090E0A0E0B0E084179507A60750
:1026B000B707D8F480910A018F3FB9F040E08091CC
:1026C0000A01481780F4842F90E0880F991FFC01BD
:1026D000E757FB4F20813181FC01E55FFE4F3183DD
:1026E00020834F5FECCF1092AA0410920A010BC016
:1026F0002D3B82E0380720F080910A018031D8F02C
:102700008FEF80930A01D0938804C0938704FF91D0
:10271000EF91DF91CF91BF91AF919F918F917F9179
:102720006F915F914F913F912F911F910F900FBE2D
:102730000F901F90189510910A0181E0810F8093EE
:102740000A01C9010E94FC08E12FF0E0EE0FFF1F13
:10275000E757FB4F91838083D6CF83E0809380003F
:102760008AE9809381008091BF0586FD05C0809134
:1027700081008064809381008FEF9FEF90938900A8
:102780008093880080916F00806280936F0008952D
:10279000CF93DF930E94520D8091D405843039F598
:1027A0008FE00E943B2AC1E0D0E0892B11F4C0E009
:1027B000D0E080E10E943B2A892B19F082E090E072
:1027C00002C080E090E08C2B9D2B8230910539F087
:1027D0008330910539F0019739F481E006C01092F9
:1027E000D40505C082E001C083E08093D405DF9169
:1027F000CF9108956F3018F086958058089589E03C
:10280000689F802D11240895A0E0B0E0EAE0F4E193
:102810000C94C52EC82F0E942229009138041091D3
:10282000390420913A0430913B046B017C01C01AB9
:10283000D10AE20AF30A9701860149E8C41643E186
:10284000D406E104F10410F010923C0460933804C3
:102850007093390480933A0490933B042091A90427
:102860008FEF820F8230D8F5E0913C04EE2309F41B
:102870004EC1E13011F482E0B8C1E03108F034C15A
:1028800081E08E0F80933C04F0E0E757FB4FC0835C
:10289000803109F0ACC1EBE8F4E0213029F4A181EA
:1028A000A695A695808108C080819181A92FA695C3
:1028B000A695A69596958795A03148F4B0E090E04E
:1028C000AA0FBB1FA55FBE4F11969C938E931092CB
:1028D000AA04329684E0E939F807F9F688C1233072
:1028E00009F005C1E0913C04E11104C0CF3009F0CA
:1028F0007EC10DC1E83148F481E08E0F80933C0425
:10290000F0E0E857FB4FC08372C1E83109F0ECC03A
:10291000C111EAC040E050E0ABE0CA01B3E0880F6B
:10292000991FBA95E1F7A49F9001A59F300D11243E
:10293000F901E757FB4F6081E1817E2F7770759534
:102940006795FC01EE0FFF1FE55FFE4F718360830B
:10295000F901E657FB4FB081B695B695B695E18182
:10296000FE2FF295FF0FF07E6F2F6B2BE695E6950D
:10297000E6957E2F777075956795FC01EE0FFF1F2A
:10298000E35FFE4F71836083F901E557FB4FB08130
:10299000B295B695B695B370C181DC2FDD0FDD0F12
:1029A0006D2F6B2BC295C695C695C370E281E17001
:1029B000EE0FEE0F7E2F7C2B75956795FC01EE0FC9
:1029C000FF1FE15FFE4F71836083F901E357FB4F07
:1029D000B081B695E181FE2FF795FF27F7956F2F10
:1029E0006B2BE6957E2F777075956795FC01EE0F42
:1029F000FF1FEF5EFE4F71836083F901E257FB4FCB
:102A0000B081B295BF70E181FE2FF295F07F6F2FFC
:102A10006B2BE295EF707E2F777075956795FC01B3
:102A2000EE0FFF1FED5EFE4F71836083F901E157EA
:102A3000FB4FB081BB1FBB27BB1FC181DC2FDD0F4C
:102A40006D2F6B2BCC1FCC27CC1FE281E370EE0FD8
:102A50007E2F7C2B75956795FC01EE0FFF1FEB5EBB
:102A6000FE4F71836083F901EF56FB4FB081B6953D
:102A7000B695E181FE2FF295FF0FFF0FF07C6F2FCF
:102A80006B2BE695E6957E2F777075956795FC0123
:102A9000EE0FFF1FE95EFE4F71836083F901EE5672
:102AA000FB4F20812295269527703181E32FEE0F71
:102AB000EE0FEE0F6E2F622B732F72957695777057
:102AC00075956795FC01EE0FFF1FE75EFE4F718362
:102AD00060834F5F5F4F4230510509F01ECF8091F8
:102AE0009F0483FF1092AA0410923C0480C02430FB
:102AF00009F07DC060913C0461110BC0C83AB1F48B
:102B0000109275051092740588EA0E94610681E0B2
:102B10006CC0613019F4C093370404C0623031F4E2
:102B2000C09336048C2F0E9461065AC0E09136048F
:102B30002E2F30E0220F331F462F50E0C90102969E
:102B4000841795073CF0633268F7FA01EA57FB4FA8
:102B5000C083E8CF2D5F3F4F8C2F90E060917405CC
:102B6000709175054217530749F4982F88278627D7
:102B70009727909375058093740532C0681779077D
:102B800069F580913704813049F5E13118F080E131
:102B900080933604F0903604CAE8D4E000E010E0F8
:102BA0000F15D0F4FE013197808190E0982F88278F
:102BB0002881822B63E0969587956A95E1F70E94BC
:102BC000FC08F801EE0FFF1FE55FFE4F9183808345
:102BD0000F5F1F4F2296E4CF1092AA0410923C047C
:102BE00080913C04882319F08F5F80933C04CDB71B
:102BF000DEB7E8E00C94E12ECF93DF93E82FF0E00E
:102C0000E654FA4FE185E03150F4F894F0E0EE0F2D
:102C1000FF1FE55FFE4F80819181789437C0E131DD
:102C200031F0E23141F0E03161F582E101C083E150
:102C30000E94642A2BC08FE00E943B2AC1E0D0E0B2
:102C4000892B11F4C0E0D0E080E10E943B2A892B5F
:102C500019F082E090E002C080E090E08C2B9D2B88
:102C60008230910541F08330910541F0019761F088
:102C700086EA92E00BC08CE090E008C089E591E024
:102C800005C080E092E002C084EF93E0DF91CF9135
:102C90000895A2E2B0E0EFE4F6E10C94BB2E9E01B1
:102CA0002F5F3F4F80E1D9011D928A95E9F764E0DB
:102CB00072E082EE95E029A33AA30E940E2B0E94B7
:102CC000AE0B1D8A1E8A1F8A188E312C212C00E023
:102CD000812C912C540170EC472E7DE9572E78E51C
:102CE000672E75E3772EE0E5CE2EE3ECDE2EE12CA9
:102CF000F12C84EF91E0A0E0B0E08D8F9E8FAF8F3C
:102D0000B8A380EC97EFAAEBB7E3898F9A8FAB8FCC
:102D1000BC8F80EC9DE9A8E5B5E3898B9A8BAB8BE2
:102D2000BC8B82EE95E00E94222C892B09F4E1C035
:102D300082EE95E00E944F2C9C0133272C32310506
:102D400009F442C0ACF42332310509F0ABC019825A
:102D50001A821B821C821D821E821F82188619867F
:102D60001A861B861C861D861E861F86188A60C0D2
:102D70002434310529F02335310509F4B2C092C05D
:102D800064E482EE95E00E94E02A2AE030E040EC24
:102D90005DE968E575E382EE95E00E946E2B6CE2DA
:102DA00082EE95E00E94E02A2AE030E040EC57EF06
:102DB0006AEB77E382EE95E00E946E2B6CE282EE86
:102DC00095E00E94202BADCF0F5F043009F0A9CF12
:102DD00029813A814B815C81A8EEB3E00E94432EA9
:102DE000698B7A8B8B8B9C8B2D813E814F81588593
:102DF0000E94432E698F7A8F8B8F9C8F29853A850D
:102E00004B855C852D8F3E8F4F8F58A32D853E853A
:102E10004F8558890E94432E6B017C0160323EE44D
:102E200073078105910530F462E38CE10E94BD09CE
:102E300000E077CF603345E774078105910510F412
:102E400062E2F3CF60345CE975078105910510F407
:102E500066E2EBCF80E5C81683ECD806E104F10406
:102E600010F462E1E2CF90E6C9169AEED906E104C9
:102E7000F10410F465E1D9CFA0E7CA16A1E1DA06A2
:102E8000A1E0EA06F10410F461E0CFCFB0EACB167E
:102E9000B6E8DB06B1E0EB06F10410F463E0C5CF61
:102EA00065E0C3CF10ED180F1A3008F03ACFE1E01B
:102EB000F0E0EC0FFD1F24E0029FE00DF11D112456
:102EC0002081318142815381AAE0B0E00E94432EEB
:102ED000610F711D811D911D6083718382839383B6
:102EE00020CF49885A886B887C88812C912C54018A
:102EF00018CF81149104A104B10489F4C301B20173
:102F00000E942C0A61E070E080E090E00E94452978
:102F10001D8A1E8A1F8A188E312C22242A948D8D98
:102F20009E8DAF8DB8A188169906AA06BB06D0F46F
:102F30000E94E6092D893E894F89588D280F311D41
:102F4000411D511D2D8B3E8B4F8B588F381608F429
:102F5000382E821508F4282E3FEF831A930AA30A0D
:102F6000B30A56C0C301B20128EE33E040E050E09E
:102F70000E947A2EBA01A9012AE030E082EE95E0A3
:102F80000E94C52B6CE282EE95E00E94E02A4AE0A6
:102F900050E0632D82EE95E00E94D42B6CE282EE2D
:102FA00095E00E94E02A6D897E898F89988DA50120
:102FB00094010E947A2EBA01A9012AE030E082EE43
:102FC00095E00E94C52B6CE282EE95E00E94E02A1B
:102FD0004AE050E0622D82EE95E00E94D42B6CE234
:102FE00082EE95E00E94202B4C0C5D1C6E1C7F1C19
:102FF000898D9A8DAB8DBC8D84159505A605B70579
:1030000020F449885A886B887C88812C912C540143
:1030100029893A894B895C89283E3340410551050D
:1030200009F07FCEA296E2E10C94D72EACE1B0E09D
:10303000ECE1F8E10C94C52E0E9422296B017C0181
:1030400081E00E949C0A14E703E0198361E0CE014D
:1030500001960E940D0C009373050E948B0B6AEF82
:1030600070E080E090E00E944529809173058330F4
:1030700089F482EE95E00E94222C892B59F40E945B
:1030800022296C197D098E099F096038734C894C7F
:103090009140D8F280917305833009F44FC08FE7D7
:1030A0000E9495090E94A8098983843511F083E064
:1030B0005CC00E94A80910924605809347050E94B3
:1030C000A8092091460530914705280F311D3093FE
:1030D0004705209346050E94A809809348050E9451
:1030E000A80980934905813110F7F12C0F2D10E0CC
:1030F0008091490590E0880F991F0817190740F43F
:103100000E94A809F801E65BFA4F8083F394EECFA2
:1031100080E7898361E0CE0101960E940D0C83E077
:10312000809373050E948B0B62E370E080E090E077
:103130000E94452980917305833011F482E015C007
:103140008FE70E9495090E94A8098983803509F0BC
:10315000AECF0FE915E00E94A809F80181938F0115
:10316000F5E00A3B1F07B9F781E06C96E8E00C94A4
:10317000E12E80914505992787FD9095A92FB92FBC
:10318000FC013196EB30F10508F066C0EC5CFF4FB6
:103190000C94F22E62E778E082EE95E00E94FC2A21
:1031A00080E893E00E94620C6AE578E082EE95E0A8
:1031B0000E94FC2A65E378E082EE95E00E94FC2AFA
:1031C0006BE078E082EE95E00E94FC2A6AEE77E000
:1031D00082EE95E00E94FC2A6DEB77E082EE95E0AE
:1031E0000E94FC2A67E977E082EE95E00E94FC2AC3
:1031F00063E777E082EE95E00E94FC2A6CE477E0DA
:1032000082EE95E00E94FC2A82EE95E00E94E82A78
:103210000E94930D21C06FE277E01AC06AE077E068
:1032200017C065EF76E014C066ED76E011C062E984
:1032300076E00EC06DE776E00BC068E676E082EEE1
:1032400095E00E94FC2A62E276E002C06CE076E043
:1032500082EE95E00E94FC2A6AE070E080E090E057
:103260000E94452982EE95E00E94222C892B29F0AC
:1032700082EE95E00E944F2CF5CF0895ACE1B0E0CE
:10328000E4E4F9E10C94C52E909145059F3F09F0C7
:1032900023C1482F50E0FA013A97EF36F10508F0C4
:1032A0000FC1E15CFF4F0C94F22E61E172E0A0C00F
:1032B0006DE172E082EE95E00E940E2B85E7898336
:1032C0008BE1EFE9F5E0DE01129601900D928A950F
:1032D000E1F76CE1CE0101960E940D0C0E948B0B70
:1032E00083E08093730568EC70E080E090E00E94DA
:1032F000452980917305843009F0E2C08FE70E9470
:1033000095090E94A8098983853509F0D9C06DEE19
:1033100074E082EE95E00E94FC2A6FEC74E082EE8D
:1033200095E00E94FC2A61EB74E096C065E372E0D0
:1033300082EE95E00E940E2B89E6898361E0CE0142
:1033400001960E940D0C0E948B0B83E08093730505
:1033500068EC70E080E090E00E9445298091730560
:10336000843009F0ADC08FE70E9495090E94A8093A
:1033700089838E010E5F1F4F7E014DE1E40EF11C2B
:103380000E94A809F80181938F01EE15FF05C1F78E
:103390008BE1FE013296AFE9B5E001900D928A957E
:1033A000E1F78981893409F08BC063E974E082EE2A
:1033B00095E00E94FC2A65E774E082EE95E00E94A9
:1033C000FC2A67E574E048C06FE472E082EE95E0A5
:1033D0000E940E2B8EEF8093450572C0805287505D
:1033E000805390914805981708F066C06EE572E02A
:1033F00082EE95E00E940E2B63C084E18093450528
:1034000060E274E029C085E18093450569EE73E0D0
:1034100023C086E18093450562EB73E01DC087E120
:103420008093450568E673E017C088E18093450501
:1034300067E573E011C089E18093450563E473E0BB
:103440000BC08AE1809345056EE273E005C08BE115
:103450008093450566E073E082EE95E00E94FC2AC9
:103460002FC06CEE72E082EE95E00E94FC2A809103
:10347000AD0591E01DC066ED72E082EE95E00E9420
:10348000FC2A8091AD0592E013C061EC72E082EEFF
:1034900095E00E94FC2A8091AD0594E009C066EA9F
:1034A00072E082EE95E00E94FC2A8091AD0598E0E2
:1034B00089278093AD058FEF809345050E943410D6
:1034C00082EE95E00E94222C892B09F45BC182EEEA
:1034D00095E00E944F2CF4CF0E943311882309F409
:1034E00051C18091DF04811104C08FEF80934505A5
:1034F00041C140E050E060E070E080EE94E00E9466
:10350000692F40914505042F112707FD1095212FA4
:10351000312FF8013197EB31F10508F01BC1E2556D
:10352000FF4F0C94F22E552747FD509520914805EA
:1035300030E0241735070CF40DC18B019C010150BC
:10354000110921093109003211052105310558F011
:10355000C0904905EBE4F5E0F12CD12CA8E2EA2E6D
:10356000415051090FC0FA01E156FA4F6150608392
:10357000D9C0DF0111972C9130E02417350729F0CD
:10358000F3943296FC10F5CFCBC00E2D10E020E066
:1035900030E0061717072807390741F42081DA01C0
:1035A000A156BA4F11962C93DD24D394E394E8CF1F
:1035B0006F3F71058105910511F008F0CBC0609354
:1035C000B705B0C06F3F71058105910511F008F096
:1035D000C1C06093B805A6C06F3F71058105910514
:1035E00011F008F0B7C06093B9059CC02091E004C9
:1035F00020622037E9F440E050E060E070E081EEC6
:1036000094E00E94692F9B01AC01DC01CB01019782
:10361000A109B1090897A105B10508F0AEC0A4ED54
:10362000B0E30E94432E6A5E7C4A8A46954E24C0CF
:103630002636E9F440E050E060E070E081EE94E08E
:103640000E94692F9B01AC01DC01CB010197A1090C
:10365000B1090797A105B10508F08FC0A8EAB1E646
:103660000E94432E645E7C438E46944E05C06115D5
:1036700071058105910579F08B019C01005C1D4964
:10368000284535430130FAE51F07F2E62F07F2E03F
:103690003F0708F05FC06093AF057093B00580935B
:1036A000B1059093B2053EC06F3F7105810591054C
:1036B00011F008F04FC06093B30534C08B019C013A
:1036C00001501109210931090F3F1105210531056B
:1036D00008F040C06093B40525C08B019C01045CD8
:1036E0001940210931090D344DE114072105310537
:1036F00028F47093B6056093B50514C06115710583
:103700008105910521F48FEF8093AE050BC06134E4
:10371000710581059105F0F461506093AE0502C01A
:10372000DD20C1F08091DE0481111AC080917F05F7
:1037300090918005A0918105B09182050196A11D0F
:10374000B11D80937F0590938005A0938105B09370
:10375000820506C060E772E082EE95E00E940E2BC3
:103760000E9429118FEF809345056AE082EE95E073
:103770000E94202B0E94341005C061E070E080E0C0
:1037800090E07ACF6C96E8E00C94E12E6AE572E066
:1037900082EE95E00E94FC2A62E472E082EE95E0FF
:1037A0000E94FC2A82EE95E00E94222C892B31F0A7
:1037B00082EE95E00E944F2C0E943E190E9416183E
:1037C000823029F0833051F46DE072E002C064E28F
:1037D00072E082EE95E00E94FC2A08958FEF8093BC
:1037E00045051092DE040E943410809145058E3FFD
:1037F00069F082EE95E00E94222C892BB1F382EED3
:1038000095E00E944F2C0E943E19EFCF08950F9330
:103810001F93109145051F3F09F0D2C0893409F468
:1038200057C000F5883309F469C058F4803309F4AF
:1038300077C008F061C08B3109F440C08132B1F12A
:10384000B9C0813409F487C030F4893309F466C003
:10385000803461F1AFC0823409F48EC0863409F43B
:1038600048C0A8C0823609F487C078F4883531F1A1
:1038700028F48235C1F18335E1F09CC08A3509F422
:1038800094C0813609F467C095C0823761F128F48D
:10389000863679F18936E1F08DC0883779F08A373C
:1038A00009F483C0833709F085C003C061E172E089
:1038B00015C00E94640D6EE872E004C00E946D0D98
:1038C00068EA72E082EE95E00E940E2B8EEF70C0E7
:1038D0000E947A060E94BF0667EC72E082EE95E0D5
:1038E0000E940E2B67C081E00E94DF0660EE72E04E
:1038F000F5CF0E94DE105EC080535AC06AEF71E0BF
:1039000082EE95E00E94FC2A90919E0588E0890F46
:103910008871977E892B80939E051AC089E048C0E4
:1039200067EE71E082EE95E00E94FC2A8091BF056F
:103930009091C005A091C105B091C20520E18227F8
:103940008093BF059093C005A093C105B093C205B5
:10395000109345052FC061ED71E082EE95E00E9465
:10396000FC2A8091BF059091C005A091C105B0913E
:10397000C20540E4842710C060EC71E082EE95E05F
:103980000E94FC2A8091BF059091C005A091C105BD
:10399000B091C20520E282278093BF059093C005B5
:1039A000A093C105B093C20502C00E94C61B8FEF51
:1039B00080934505809145058E3F09F0D4C0DDC058
:1039C0000E943311882309F4D8C08091DF0481114B
:1039D00004C08FEF80934505C6C040E050E060E032
:1039E00070E080EE94E00E94692F00914505112758
:1039F00007FD1095212F312FF8013197E930F1059E
:103A000008F0B4C0E753FF4F0C94F22E8B019C01D9
:103A1000015C1D49284535430F3F19452246324078
:103A200008F0A4C060937B0570937C0580937D05AE
:103A300090937E0577C060937F0570938005809397
:103A400081059093820581E08093DE046BC068302D
:103A500071058105910508F089C06093830562C0F6
:103A60008B019C0101501109210931090A3011050E
:103A70002105310508F07AC06093840553C061EBDD
:103A800071E080EE94E00E94A33010E0009799F07E
:103A90000E947D30009779F0183130F4E12FF0E08A
:103AA000EA58FA4F87871F5F61EB71E080E090E092
:103AB0000E94A330EBCF1831A8F5E12FF0E0EA58CF
:103AC000FA4F17861F5FF7CF6530710581059105A5
:103AD00008F04CC060939D0525C08B019C010150EE
:103AE0001109210931090630110521053105F0F5CB
:103AF00020919E05287F262B20939E0513C08B01C5
:103B00009C0101501109210931090115124C214074
:103B1000310560F56093770570937805809379059A
:103B200090937A058091DE04811113C080917F0506
:103B300090918005A0918105B09182050196A11D0B
:103B4000B11D80937F0590938005A0938105B0936C
:103B500082050E9429118FEF809345056AE082EE6D
:103B600095E00E94202B0E94B91807C060E772E020
:103B700082EE95E00E940E2BECCF1F910F910895DD
:103B80008FEF809345051092DE040E94B918809152
:103B900045058E3F69F082EE95E00E94222C892B2C
:103BA000B1F382EE95E00E944F2C0E94071CEFCFEC
:103BB0006AE070E080E090E00E94452982EE95E0A6
:103BC0000E94222C892B29F082EE95E00E944F2C36
:103BD000F5CF0895CF93C82F682F82EE95E00E940D
:103BE0007C2C90916A059C2790936A05CF9108954B
:103BF000A1E0B0E0EEEFFDE10C94CB2E99830E94A2
:103C0000EA1D9981892F0E94EA1D2196E2E00C9419
:103C1000E72E1F93CF93DF93182FEB0110926A05C5
:103C200065EB70E082EE95E00E94590662E670E076
:103C300082EE95E00E945906812F0E94EA1DCE0176
:103C40000E94F81DDF91CF911F91089560916A0540
:103C500082EE95E00E947C2C0895A1E2B0E0E3E3BF
:103C6000FEE10C94C72E7B018A018C3009F453C10C
:103C700008F040C0863009F4BCC018F5833009F460
:103C800091C070F4813009F472C0823009F048C2EA
:103C90006BE170E082E00E94091E0FE915E078C038
:103CA000843009F487C0853009F03AC26091490533
:103CB00070E0660F771F85E00E94091E0AE415E098
:103CC00086C0893009F4A7C070F4873009F49BC01E
:103CD000883009F025C261E070E088E00E94091E8A
:103CE0008091D40523C28A3009F4CAC08B3009F40C
:103CF000F2C016C28A3609F475C1D8F4873609F4C1
:103D00003AC138F4853609F40EC1863609F41FC16C
:103D100007C2883609F437C1893609F001C261E06B
:103D200070E089E60E94091E0E947A060E94BF0682
:103D3000F5C18D3609F4D4C138F48B3609F491C13C
:103D40008C3609F49AC1ECC18E3609F4DCC1873C8B
:103D500009F0E6C161E070E087EC0E94091E81E095
:103D60000E94EA1D0E94261E10926B05E3C169E2C3
:103D700070E081E00E94091E06E715E0F8018191DC
:103D80008F010E94EA1DF5E00F391F07B9F7D0C176
:103D9000F80181918F010E94EA1DF5E00A3B1F079F
:103DA000B9F7C6C161E070E083E00E94091E0E947D
:103DB0001618BCC161E070E084E00E94091E81E039
:103DC0000E94EA1D0E94261E0E944916B3C18091DE
:103DD000490590E0880F991F98012A54354028170B
:103DE000390708F0A5C1F80181918F010E94EA1DF1
:103DF000EECF62E070E086E00E94091E80E893E06A
:103E00000E94F81D95C161E070E087E00E94091EE4
:103E1000809148058BC186E6898361E0CE010196D9
:103E20000E940D0C0E948B0B83E08093730568EC5D
:103E300070E080E090E00E94452980917305843015
:103E4000D9F48FE70E9495090E94A80989838634D6
:103E500069F460E270E089E00E94091E10E20E94AD
:103E6000A8090E94EA1D1150D1F762C161E070E01B
:103E700089E00E94091E52C161E070E089E053C1EF
:103E800069E170E08AE00E94091E82E08093BA0531
:103E9000209172058091BF059091C005A091C10548
:103EA000B091C205222311F0806801C08F77809302
:103EB000BF059093C005A093C105B093C2050AEB5E
:103EC00015E0F80181918F010E94EA1DF5E0033DA4
:103ED0001F07B9F72DC161E270E08BE00E94091E57
:103EE0008091AA048F3F39F08091AA0491E0980F45
:103EF0009093AA0402C08091AA040E94EA1D10E0D7
:103F0000812F0E94FC150E9427090E94F81D1F5F47
:103F10001031B1F70DC161E070E08CE00E94091E24
:103F20008091D30503C161E070E085E60E94091E1F
:103F300089E2E816F10409F0F8C0D801E6E7F5E0F7
:103F40008D91819385E0EF39F807D1F7E7C061E003
:103F500070E086E60E94091EEBE1EE16F10409F01E
:103F6000E4C0D801EFE9F5E08D91819385E0EA3B6B
:103F7000F807D1F7D3C061E070E087E60E94091E20
:103F80000E94640DCBC061E070E088E60E94091ECB
:103F900085E789838BE1EFE9F5E0DE011296019078
:103FA0000D928A95E1F76CE1CE0101960E940D0C0D
:103FB0000E948B0B83E08093730560E273E080E0E6
:103FC00090E00E94452980917305843009F0ADC0CE
:103FD0008FE70E9495090E94A8098983853509F019
:103FE000A4C09CC061E070E08AE60E94091E89E6D8
:103FF000898361E0CE0101960E940D0C0E948B0B1B
:1040000083E08093730560E273E080E090E00E94BB
:10401000452980917305843009F087C08FE70E949D
:1040200095090E94A80989838E010E5F1F4F7E01AA
:10403000EDE1EE0EF11C0E94A809F80181938F01B9
:10404000EE15FF05C1F78BE1FE013296AFE9B5E051
:1040500001900D928A95E1F78981893409F065C054
:104060005DC061E070E08BE60E94091EF80180816E
:104070008093D4050E946D0D51C061E070E08CE624
:104080000E94091EF0E2EF16F10461F487E68983CD
:1040900080E2F801DE01129601900D928A95E1F717
:1040A00061E203C087E4898361E0CE0101960E944A
:1040B0000D0C0E948B0B83E0809373056CE474E01D
:1040C00080E090E00E94452980917305843069F575
:1040D0008FE70E9495090E94A809873431F51EC018
:1040E00061E070E08DE60E94091E89E1E816F104A6
:1040F000E1F4D801EAEBF5E08D91819385E0E33DB1
:10410000F807D1F70BC061E070E08EE60E94091E4F
:10411000F80180818093D3050E944D0D81E006C097
:1041200061E070E08AEC0E94091E80E00E94EA1DB6
:104130000E94261EA196E6E00C94E32EA0E0B0E0DB
:10414000E4EAF0E20C94C52ECAECD3E014E606E0F3
:1041500035E0F32E44E0E42E53E0D52E62E0C62E87
:1041600082EE95E00E94222C892B09F49BC082EEFE
:1041700095E00E944F2C282F809335044091340401
:1041800050E04730510560F7FA01EE52FF4F0C94B2
:10419000F22E853B29F781E080933404E1CF82360B
:1041A00009F07DC0C0923404DBCF80933304809348
:1041B0003204D0923404D4CF9C013327309331049D
:1041C0002093300490913204982790933204E09227
:1041D0003404C6CF382F2227409130045091310447
:1041E000242B352B309331042093300490913204EA
:1041F000982790933204F09234042536310508F460
:10420000AFCF61E070E08CEC0E94091E81E00E945B
:10421000EA1D0E94261E43C020912E0430912F04D7
:10422000F901E653FC4F80839091320498279093D4
:104230003204C901019690932F0480932E0420919B
:104240003004309131048217930708F489CF00932A
:10425000340486CF8091320482130BC060912E0407
:1042600070912F044AEC53E0809133040E942D1E7C
:104270000DC062E070E08BEC0E94091E8091330457
:104280000E94EA1D80916A050E94EA1DFE01812FAD
:1042900011928A95E9F710922F0410922E04109231
:1042A00034045ECFCDB7DEB7E8E00C94E12E81E0B8
:1042B00080936B0580916B05882349F082EE95E031
:1042C0000E94222C892BB1F30E949E20F3CF0895E7
:1042D000AAE2B0E0EEE6F1E20C94C32E0E941629A9
:1042E0006B017C0181E00E949C0A82EE95E00E94B5
:1042F000222C892B29F082EE95E00E944F2CF5CFDD
:104300005E9811E072E6B72EE9E2AE2E03E00E945D
:1043100016296C197D098E099F09693C7105810573
:104320009105D0F11123C1F10E9416296B017C0186
:104330005D9A80ED97E00E94AE07B982E6E7F5E06E
:10434000DE0112968A2D01900D928A95E1F76AE2BC
:10435000CE0101960E940D0C5D9880E090E00E94D5
:10436000AE07009373050E948B0B62E370E080E060
:1043700090E00E94452980917305843061F4009398
:1043800073058FE70E9495090E94A80911E0823405
:1043900019F410E001C011E08EE00E943B2A892B45
:1043A00081F411E00EC05E9A5D9A82EE95E00E9463
:1043B0004F2C8D309105A9F05CF40A9791F05E982E
:1043C0005D9882EE95E00E94222C892B61F79FCFA9
:1043D0008332910579F08234910589F70E94572143
:1043E000EECF62EB71E082EE95E00E94FC2A0E9423
:1043F000C01DE5CF0E944916E2CF8F929F92AF92E7
:10440000BF92CF92DF92EF92FF921F93CF93DF93F1
:104410008EE00E943B2A892B09F089C068EC70E08D
:1044200080E090E00E94452980E090E00E94AE0785
:104430000E9416294B015C016B017C0180ECC80EC7
:1044400082E1D81EE11CF11C0E9416296C157D0525
:104450008E059F0530F48EE00E943B2A892BA1F344
:1044600064C08EE00E943B2A892B09F05EC080ED7B
:1044700097E00E94AE070E9416296B017C01D0E0F4
:10448000C1E088E4880E86E2981EA11CB11C11E0F0
:104490008EE00E943B2A892B21F58C149D04AE04EA
:1044A000BF0430F480ED97E00E94AE07D1E0F0CF7A
:1044B0000E9416296C197D098E099F09693C7105B6
:1044C0008105910528F30E9416296B017C01C12703
:1044D00019F080ED97E002C080E090E00E94AE0706
:1044E000D7CF80E090E00E94AE07DD23B9F0809145
:1044F000D30590E0019665E070E00E94662E8093FF
:10450000D3050E944D0D0E94C8130E946D0D64EFEB
:1045100071E080E090E00E94452909C080E00E949F
:10452000DF060E94E5110E94640D0E946821DF9160
:10453000CF911F91FF90EF90DF90CF90BF90AF9001
:104540009F908F900895CF92DF92EF92FF9280E03C
:104550000E94F8070E94CF0761E089E00E94CF29FE
:1045600060E089E00E94082A61E086E00E94CF298D
:1045700061E085E00E94CF2960E08EE00E94CF29B3
:1045800060E08FE00E94CF2961E08FE00E94082A5E
:1045900060E080E10E94CF2961E080E10E94082A6A
:1045A00060E088E00E94CF2961E088E00E94082A4C
:1045B00061E081E10E94CF2960E081E10E94082A48
:1045C0000E949F0740E052EC61E070E082EE95E0CF
:1045D0000E946A2D0E94C8130E946D0D0E94AD13A7
:1045E0008FEF8093AA040E94E40778940E94162912
:1045F0006B017C018091AA048F3F59F40E94162917
:104600006C197D098E099F09603D774081059105F0
:1046100088F380ED97E00E94AE0761E08EE00E9493
:10462000082A5E9A82EE95E00E94222C892B29F0BE
:1046300082EE95E00E944F2CF5CF6DEF72E082EE96
:1046400095E00E94DD2A80E893E00E94620C64E11C
:1046500073E082EE95E00E94DD2A4AE050E064E0DB
:1046600070E082EE95E00E94AD2B62E370E080E0A6
:1046700090E00E94452982EE95E00E94222C04974A
:104680000CF182EE95E00E944F2C82349105D1F41A
:1046900082EE95E00E944F2C8E34910599F482EEC3
:1046A00095E00E944F2C8434910561F482EE95E0F0
:1046B0000E944F2C819731F480E090E00E94AE0779
:1046C0000E946821409177055091780560917905A5
:1046D00070917A05DB01CA010197A109B10904971C
:1046E000A105B10568F44093A904433029F440EAD8
:1046F00056E861E070E004C040E052EC61E070E038
:1047000082EE95E00E946A2D0E94FD215E9880E075
:1047100090E00E94AE070E94AD131092C5048091F4
:10472000BF0583FF11C080918B05882351F08091D4
:104730009205882331F080919905882311F087E054
:1047400001C085E08093C50480E00E949C0A8091AE
:10475000C6040E94D0090E948B0B10923F04109255
:104760003E0410923D04F12C8091D4058F15B0F0D9
:1047700062E370E080E090E00E94452980ED97E0E0
:104780000E94AE0762E370E080E090E00E9445295D
:1047900080E090E00E94AE07F394E6CF80919E0502
:1047A00084FF08C0982F987181E0983109F080E06B
:1047B0000E94A1118FE00E94F807FF90EF90DF9018
:1047C000CF900895EF92FF920F931F93CF93DF93B3
:1047D0008C016EE770E082EE95E00E945906E801D8
:1047E000F12CF0E2EF2E8E0188818D57823048F453
:1047F0006DE770E082EE95E00E94590688818E2573
:1048000088832196F801608182EE95E00E947C2CDD
:10481000F394F9E0FF12E7CF6EE770E082EE95E0E7
:104820000E945906CDB7DEB7E6E00C94E32EA9E06E
:10483000B0E0EDE1F4E20C94CB2E9091C70491111D
:104840000EC09EEF99838A836B8350E05595479500
:104850004C832D83198618861F821E822EC040919C
:10486000CC04842F90E0B4E095958795BA95E1F754
:10487000242F2F7030E08217930719F18DEF898371
:104880001B82FE01349650E0842F90E0A4E09595C1
:104890008795AA95E1F7242F2F7030E082179307B0
:1048A00049F0DC01A353BB4F8C918193405F5F5F64
:1048B000563051F74093CC045A83CE0101960E94A2
:1048C000E2238091C70490E0019666E070E00E94C8
:1048D000662E8093C7042996E2E00C94E72EA0E0B0
:1048E000B0E0E5E7F4E20C94C42E6C016EE770E0F2
:1048F00082EE95E00E9459068601E12CF12CC0E081
:10490000D0E030E2B32EF801608183E8860F823078
:1049100078F46DE770E082EE95E00E945906F801A8
:1049200060816B2570E082EE95E00E94590604C01C
:1049300082EE95E00E947C2CE114F10459F0F8011C
:1049400080819E01280F311DC901C92FDD27C80FA5
:10495000D91FDD273FEFE31AF30A89E0E816F104D7
:1049600059F028E0E216F10421F48C2F8095F6012D
:1049700080870F5F1F4FC7CFCDB7DEB7E9E00C943C
:10498000E02EA9E0B0E0E7ECF4E20C94CB2EE82FA7
:10499000362F8091C70490E0019664E270E00E9497
:1049A000662E8093C70458E9598350E15A838130B9
:1049B00089F048F08230B9F08330D9F48B8381EFED
:1049C0008C833D8319C085E08B8381EF8C832F5FBF
:1049D0002D8312C08B8381EF8C8384E6489FA001D6
:1049E00011245D8309C084E08B8381EF8C83ED8388
:1049F00003C00E94DE1104C0CE0101960E946F2404
:104A00002996E2E00C94E72EA2E0B0E0EAE0F5E2BD
:104A10000C94C02E182F762E2A8349830E942229B7
:104A20006B017C018091DD048090C8049090C904E2
:104A3000A090CA04B090CB042A8149818823C1F098
:104A4000D701C60188199909AA09BB094C015D0162
:104A500091EE89169EE29906A104B10420F1241773
:104A600008F4422F202F672D812F0E94C12413C0EC
:104A7000D701C60188199909AA09BB094C015D0132
:104A800091E3891695E79906A104B10460F0672DBA
:104A9000812F0E941724C092C804D092C904E092CA
:104AA000CA04F092CB042296EDE00C94DC2EA2E234
:104AB000B0E0EDE5F5E20C94C12E8CE00E94B70960
:104AC00081110DC06CE173E082EE95E00E940E2B27
:104AD0005E9A80E00E949C0A0E948B0B5E9882EE98
:104AE00095E00E94222C892B01F182EE95E00E9434
:104AF0004F2C9091A904992319F00E940414EFCF30
:104B000040913E0450E09A012F5F3F4F2F713327B1
:104B100060913F0470E02617370709F3FA01E75B5D
:104B2000FB4F808320933E04DACF8091730584305D
:104B300009F086C00E942229611571058105910541
:104B400049F06093B7047093B8048093B9049093CC
:104B5000BA040CC081E090E0A0E0B0E08093B7041C
:104B60009093B804A093B904B093BA048091AD04B3
:104B70009091AE0481609093AE048093AD0483E085
:104B8000809373058FE70E94950909E614E00E945F
:104B9000A809F80181938F01F4E002371F07B9F7E4
:104BA0002091720480916904982F922796FF3BC050
:104BB00090E4922790937204982F98739833F1F4AD
:104BC00010E0212F30E080916904877090E0821717
:104BD00093074CF11F5F20919E05812F90E0FC010F
:104BE000E759FB4F24FF04C080810E94C011E9CF28
:104BF000608182EE95E00E947C2CE3CF8F7399F464
:104C000080916A048093B60480916B048093B4040D
:104C100080916C048093B30480916F0490E0909332
:104C2000AC048093AB0480913D04813019F482E0A0
:104C300080933D0480913D04833011F410923D0433
:104C40000E9422296B017C018091AF049091B004F5
:104C5000A091B104B091B2040097A105B105C9F0CB
:104C6000A7019601281B390B4A0B5B0BDA01C9011E
:104C7000883B9B40A105B10560F00E94E609809346
:104C8000B5041092AF041092B0041092B1041092C7
:104C9000B2048091BB049091BC04A091BD04B0917A
:104CA000BE0446015701881A990AAA0ABB0A86E778
:104CB00095E00E94120886169706A806B90608F421
:104CC000B1C0C092BB04D092BC04E092BD04F0928B
:104CD000BE040E9457068091AA048830A0F08091FB
:104CE000BF059091C005A091C105B091C2056CE1CE
:104CF000B695A795979587956A95D1F7892B8A2BB5
:104D00008B2B09F0BEC18091AA048F5F8093AA0407
:104D10008091B7049091B804A091B904B091BA04FD
:104D20000097A105B105F1F0C81AD90AEA0AFB0AF1
:104D300086E795E00E9412086C157D058E059F059B
:104D400008F00FC18091BF0584FD04C080ED97E09D
:104D50000E94AE071092B7041092B8041092B904E2
:104D60001092BA0490917204907C909372045091C6
:104D70003E0480913F0420913D04581709F40EC170
:104D8000223009F00BC1905890937204E0919E0577
:104D9000E770F0E0E658FC4F6081693008F0E6C04B
:104DA000615040E04613E4C080933F0487E3840FE2
:104DB00090917204892B809372044093400483E0A5
:104DC00080933D045D9A109183058091C504811103
:104DD00038C18091BF0582FD40C1812F0E94970A92
:104DE0008091C6040E94D009E0919E05E770F0E032
:104DF000E658FC4F608182E794E00E94C60B8091E8
:104E0000BF0582FD33C1E091C604EF5FE093C604A5
:104E1000E83109F433C1F0E0EA58FA4F8785882376
:104E200009F42CC10E94350C813069F580919E05F2
:104E3000887149F18091AD049091AE04880F991F5B
:104E40009093AE048093AD0483E0809373050E9439
:104E50008B0B0E9422296093AF047093B00480935F
:104E6000B1049093B204672B682B692B61F481E045
:104E700090E0A0E0B0E08093AF049093B004A093E2
:104E8000B104B093B20480919E0584FF1FC080914D
:104E9000AD049091AE048E7F0E944809182F609156
:104EA000AB048091B6040E94FA13482F612F8091C1
:104EB000B50449A30E94FA130091D405282F49A1F3
:104EC0006091B3048091B4040E9404255D988091A0
:104ED000C3048130C1F018F08230B1F1DFC08EE040
:104EE0000E943B2A892B09F0D9C081E08093C3043A
:104EF0000E9416296093BF047093C0048093C1047C
:104F00009093C204CBC08EE00E943B2A892B31F5DE
:104F10000E941629C090BF04D090C004E090C10444
:104F2000F090C2046C197D098E099F09693E734097
:104F30008105910508F4B2C082E08093C30480ED3E
:104F400097E00E94AE07AAC08EE00E943B2A892B00
:104F500009F4A4C080E090E00E94AE071092C30460
:104F60009DC080E090E00E94AE07FCCE68E019CFC3
:104F7000851709F419CF4F5F242F30E090E0F90135
:104F8000EE58FB4FDC01A75BBB4F7C917083F901AE
:104F9000E05CFB4F708301968F7104CF2430B1F435
:104FA0002091400481E494E0A3E7B4E0FC013E2FAB
:104FB000381B321718F431913D93F9CF87E3820FF4
:104FC00090917204892B80937204F9CE8091C3046E
:104FD000823069F49160909372045E9A53ECE52EEE
:104FE00055E0F52E8E010F5F1F4FB80110C05E987F
:104FF00080913D04811103C081E080933D04809144
:105000003D04833059F784E080933D04E7CFF701F6
:1050100081917F0169A37AA30E94FC15F801819315
:1050200091938F0169A17AA1F3EDEF16F5E0FF06E8
:1050300071F780919E0543E754E087700E949708BE
:10504000C1CE112309F4C5CE9091C40421E0290FEB
:105050002093C4049813BDCE1DC08FE00E943B2A4C
:10506000892B09F0BACE5E9A17E0B7CE8FE00E9486
:105070003B2A892B09F0C7CE5E98C5CE1092C60494
:10508000D1CE8091AA04883009F45E9A89E0809399
:10509000AA04C8CE1092C40411509BCEA296ECE094
:1050A0000C94DD2E8230E8F4E82FF0E0EE0FFF1FC5
:1050B000EB52FA4F71836083813041F08091690037
:1050C0008C7F842B80936900E89A08958091690011
:1050D000440F551F440F551F837F842B8093690015
:1050E000E99A08951F920F920FB60F9211242F93F1
:1050F0003F934F935F936F937F938F939F93AF9360
:10510000BF93EF93FF938091D5059091D605892B9E
:1051100029F0E091D505F091D6050995FF91EF9121
:10512000BF91AF919F918F917F916F915F914F91BF
:105130003F912F910F900FBE0F901F9018951F92C7
:105140000F920FB60F9211242F933F934F935F93BB
:105150006F937F938F939F93AF93BF93EF93FF933F
:105160008091D7059091D805892B29F0E091D7053A
:10517000F091D8050995FF91EF91BF91AF919F9163
:105180008F917F916F915F914F913F912F910F90F0
:105190000FBE0F901F9018951F920F920FB60F928F
:1051A00011242F933F938F939F93AF93BF9380913D
:1051B000DA059091DB05A091DC05B091DD05309119
:1051C000D90523E0230F2D3720F40196A11DB11D31
:1051D00005C026E8230F0296A11DB11D2093D90515
:1051E0008093DA059093DB05A093DC05B093DD0591
:1051F0008091DE059091DF05A091E005B091E10579
:105200000196A11DB11D8093DE059093DF05A0934B
:10521000E005B093E105BF91AF919F918F913F91D0
:105220002F910F900FBE0F901F9018952FB7F894E5
:105230006091DA057091DB058091DC059091DD05C8
:105240002FBF08953FB7F8948091DE059091DF0558
:10525000A091E005B091E10526B5A89B05C02F3FC0
:1052600019F00196A11DB11D3FBF6627782F892F28
:105270009A2F620F711D811D911D42E0660F771FED
:10528000881F991F4A95D1F70895CF92DF92EF9228
:10529000FF92CF93DF936B017C010E942229EB01E7
:1052A000C114D104E104F10479F00E9422296C1B9D
:1052B0007D0B683E7340A0F381E0C81AD108E10875
:1052C000F108C851DC4FECCFDF91CF91FF90EF9008
:1052D000DF90CF900895789484B5826084BD84B5C2
:1052E000816084BD85B5826085BD85B5816085BDE1
:1052F000EEE6F0E0808181608083E1E8F0E01082FA
:10530000808182608083808181608083E0E8F0E03A
:10531000808181608083E1EBF0E080818460808324
:10532000E0EBF0E0808181608083EAE7F0E080815B
:1053300084608083808182608083808181608083BB
:105340008081806880831092C1000895833081F04D
:1053500028F4813099F08230A1F008958630A9F0C8
:105360008730B9F08430D1F4809180008F7D03C004
:10537000809180008F7780938000089584B58F7727
:1053800002C084B58F7D84BD08958091B0008F7771
:1053900003C08091B0008F7D8093B0000895CF93BB
:1053A000DF9390E0FC01ED50F44F2491FC01E95FA4
:1053B000F34F8491882349F190E0880F991FFC01F5
:1053C000E15DF34FA591B4918B5D934FFC01C591C5
:1053D000D4919FB7611108C0F8948C9120958223D5
:1053E0008C93888182230AC0623051F4F8948C91A6
:1053F000322F309583238C938881822B888304C03D
:10540000F8948C91822B8C939FBFDF91CF9108955C
:10541000A1E0B0E0EEE0FAE20C94C92E282F30E0D3
:10542000F901E152F44F8491F901ED50F44F1491D8
:10543000F901E95FF34F04910023C9F0882321F0BB
:1054400069830E94A6296981E02FF0E0EE0FFF1F1B
:10545000EB5DF34FA591B4919FB7F8948C916111D6
:1054600003C01095812301C0812B8C939FBF21968F
:10547000E4E00C94E52ECF93DF93282F30E0F90180
:10548000E152F44F8491F901ED50F44FD491F901B8
:10549000E95FF34FC491CC2391F081110E94A629BA
:1054A000EC2FF0E0EE0FFF1FE55EF34FA591B491F6
:1054B0002C912D2381E090E021F480E002C080E077
:1054C00090E0DF91CF9108958E3008F08E50877074
:1054D00020919D0190E4299F90011124822B8093BB
:1054E0007C0080917A00806480937A0080917A00B9
:1054F00086FDFCCF809178002091790090E0922B7E
:105500000895A0E0B0E0E7E8FAE20C94C52E6C0143
:105510007A01EB01E60EF71E00E010E0CE15DF0584
:1055200061F06991D601ED91FC910190F081E02D3F
:10553000C6010995080F191FF1CFC801CDB7DEB715
:10554000E8E00C94E12E6115710589F0DB010D9006
:105550000020E9F7AD0141505109461B570BDC0112
:10556000ED91FC910280F381E02D0995089580E092
:1055700090E00895EF92FF920F931F93CF93DF93E4
:105580008C01FB01C0E0D0E064917F018FEFE81A4D
:10559000F80A662361F0D801ED91FC910190F08149
:1055A000E02DC8010995C80FD91FF701EDCFCE0135
:1055B000CDB7DEB7E6E00C94E32E0E94A32A08954F
:1055C000DC01ED91FC910190F081E02D09950895A9
:1055D0000F931F93CF93DF93EC016DE00E94E02ABD
:1055E0008C016AE0CE010E94E02A800F911FDF91BA
:1055F000CF911F910F9108950F931F93CF93DF9336
:10560000EC010E94BA2A8C01CE010E94E82A800F88
:10561000911FDF91CF911F910F9108950F931F93C9
:10562000CF93DF93EC010E94A32A8C01CE010E944C
:10563000E82A800F911FDF91CF911F910F9108955C
:105640000F931F93CF93DF93EC010E94E02A8C010C
:10565000CE010E94E82A800F911FDF91CF911F9108
:105660000F910895A1E2B0E0E8E3FBE20C94C12EB3
:105670007C01C42EE52FCB01D22E19A221E02D15DD
:1056800010F02AE0D22E8E010F5D1F4F8D2C912C31
:10569000A12CB12C6C2D7E2FA50194010E947A2E95
:1056A0008C2DD29E80191124015011098A3010F4DA
:1056B000805D01C0895CF8018083211531054105B9
:1056C000510521F0C22EE32FCA01E4CFB801C70172
:1056D0000E94A32AA196ECE00C94DD2EA0E0B0E09D
:1056E000E4E7FBE20C94C52EEC016A017B01211575
:1056F000310541F4E881F9810190F081E02D642FBA
:1057000009951DC02A303105A9F477FF12C06DE25A
:105710000E94E02A8C0144275527BA014C195D09E3
:105720006E097F092AE0CE010E94322B800F911F63
:1057300006C02AE0B701A601CE010E94322BCDB7E8
:10574000DEB7E8E00C94E12E9A01AB01662757FD25
:105750006095762F0E946E2B08950F931F93CF9321
:10576000DF93EC019A01AB01662757FD6095762F18
:105770000E946E2B8C01CE010E94E82A800F911F9F
:10578000DF91CF911F910F9108952115310549F4B3
:10579000DC01ED91FC910190F081E02D642F0995E1
:1057A00008950E94322B08959A01462F50E060E040
:1057B00070E00E94C52B08959A01AB0160E070E093
:1057C0000E94C52B08950F931F93CF93DF93EC0195
:1057D0000E94C52B8C01CE010E94E82A800F911FE8
:1057E000DF91CF911F910F9108950F931F93CF9346
:1057F000DF93EC019A01AB0160E070E00E94C52BE1
:105800008C01CE010E94E82A800F911FDF91CF9179
:105810001F910F9108950F931F93CF93DF93EC0186
:105820009A01462F50E060E070E00E94C52B8C0189
:10583000CE010E94E82A800F911FDF91CF911F9126
:105840000F910895FC0124853585F901E05CFF4F37
:1058500080819181F901EE5BFF4F20813181821BB4
:10586000930B8F7399270895FC0184859585FC011E
:10587000E05CFF4F40815181FC01EE5BFF4F2081D6
:1058800031814217530741F00190F081E02DE80F7C
:10589000F91F808190E008958FEF9FEF0895FC013C
:1058A00084859585FC01E05CFF4F40815181FC01BE
:1058B000EE5BFF4F208131814217530779F0A081C1
:1058C000B181A80FB91F8C91208131812F5F3F4F8B
:1058D0002F7333273183208390E008958FEF9FEF5C
:1058E0000895FC0181A1882329F0A489B5898C91B0
:1058F00086FFFBCF11A20895CF93DF93FC0126858D
:105900003785D901A05CBF4F8D919C91119701966D
:105910008F739927E901CE5BDF4F48815981841746
:105920009507D9F30D90BC91A02DA20FB31F6C93D6
:10593000A685B785A05CBF4F11969C938E93A689D0
:10594000B7892C9181E090E0078C02C0880F991FE5
:105950000A94E2F7282B2C9381E081A30488F5892F
:10596000E02D80818064808381E090E0DF91CF91A1
:10597000089508951F920F920FB60F9211242F933E
:105980003F934F938F939F93EF93FF938091C0002A
:1059900082FD1CC04091C6008091880690918906C6
:1059A00001968F73992720918A0630918B06821772
:1059B000930771F0E0918806F0918906E85BF94F52
:1059C0004083909389068093880602C08091C60028
:1059D000FF91EF919F918F914F913F912F910F9058
:1059E0000FBE0F901F90189582EE95E00E94222C1A
:1059F000892B11F00E94B92C08951F920F920FB6B7
:105A00000F9211242F933F938F939F93EF93FF93C4
:105A100020914406309145068091460690914706B4
:105A20002817390731F48091C1008F7D8093C10020
:105A300014C0E0914606F0914706EC5FF94F2081D3
:105A4000809146069091470601968F73992790930F
:105A50004706809346062093C600FF91EF919F91E1
:105A60008F913F912F910F900FBE0F901F9018951F
:105A7000A0E0B0E0EEE3FDE20C94C12EFC01138245
:105A8000128288EE93E0A0E0B0E084839583A68341
:105A9000B7838CEB93E09183808375876487578706
:105AA0004687318B208B138B028BF58AE48AD78A49
:105AB000C68AB18EA08E938E828E8F85848F8889C0
:105AC000858F8989868F8A89878F8B8980A3ECE06F
:105AD0000C94DD2ECF92DF92EF92FF92CF93DF9363
:105AE000EC016A017B01411581EE580761057105E2
:105AF000F9F0EC89FD8981E090E008A002C0880FF0
:105B0000991F0A94E2F7808360E079E08DE390E0EA
:105B1000A70196010E947A2E2150310941095109AD
:105B20005695479537952795211580E1380798F0C8
:105B3000EC89FD89108260E874E88EE190E0A701AD
:105B400096010E947A2E215031094109510956953A
:105B5000479537952795E889F9893083EA89FB8944
:105B6000208319A2EE89FF89408181E090E09C01A9
:105B70000C8C02C0220F331F0A94E2F7422B4083A1
:105B8000EE89FF8940819C010D8C02C0220F331FDA
:105B90000A94E2F7422B4083EE89FF8940819C0101
:105BA0000E8C02C0220F331F0A94E2F7422B40836F
:105BB000EE89FF8920810F8C02C0880F991F0A94FB
:105BC000E2F7809582238083DF91CF91FF90EF9061
:105BD000DF90CF9008958F929F92AF92BF92CF9215
:105BE000DF92EF92FF920F931F9381E08F9385E0F6
:105BF0008F9387E08F9383E08F9384E08F93E6EC1D
:105C00008E2E912CF2ECAF2EB12CA1ECCA2ED12C01
:105C1000B0ECEB2EF12C04EC10E025EC30E044E08D
:105C200056E068E476E082EE95E00E94382D0F9011
:105C30000F900F900F900F901F910F91FF90EF908A
:105C4000DF90CF90BF90AF909F908F9008950E946B
:105C50006B290E94A322C4EFDCE20E945725209703
:105C6000E1F30E94F42CF9CFA29FB001B39FC001D1
:105C7000A39F700D811D1124911DB29F700D811D78
:105C80001124911D08950E94342EA59F900DB49F5C
:105C9000900DA49F800D911D11240895B7FF0C94C1
:105CA000432E0E94432E821B930B0895DB018F939A
:105CB0009F930E94432EBF91AF91A29F800D911D93
:105CC000A39F900DB29F900D1124089597FB072E6E
:105CD00016F4009407D077FD09D00E94F82E07FC37
:105CE00005D03EF4909581959F4F089570956195EC
:105CF0007F4F0895A1E21A2EAA1BBB1BFD010DC008
:105D0000AA1FBB1FEE1FFF1FA217B307E407F5076B
:105D100020F0A21BB30BE40BF50B661F771F881F47
:105D2000991F1A9469F760957095809590959B01DD
:105D3000AC01BD01CF010895052E97FB1EF4009420
:105D40000E94B32E57FD07D00E947A2E07FC03D085
:105D50004EF40C94B32E50954095309521953F4FBD
:105D60004F4F5F4F089590958095709561957F4F47
:105D70008F4F9F4F08952F923F924F925F926F9255
:105D80007F928F929F92AF92BF92CF92DF92EF92CB
:105D9000FF920F931F93CF93DF93CDB7DEB7CA1B4C
:105DA000DB0B0FB6F894DEBF0FBECDBF09942A8877
:105DB000398848885F846E847D848C849B84AA841F
:105DC000B984C884DF80EE80FD800C811B81AA81AC
:105DD000B981CE0FD11D0FB6F894DEBF0FBECDBF77
:105DE000ED010895EE0FFF1F0590F491E02D099449
:105DF000AA1BBB1B51E107C0AA1FBB1FA617B707F1
:105E000010F0A61BB70B881F991F5A95A9F780950C
:105E10009095BC01CD0108958F929F92AF92BF9251
:105E2000CF92DF92EF92FF92CF93DF93EC016881E4
:105E300079818A819B81611571058105910521F424
:105E400064E279ED8BE597E02DE133EF41E050E03E
:105E50000E949C2E49015A019B01AC01A7EAB1E4C2
:105E60000E94432E6B017C01ACEEB4EFA5019401BE
:105E70000E94512EC60ED71EE81EF91EF7FE06C060
:105E800081E0C81AD108E10880E8F80AC882D982FE
:105E9000EA82FB82C701B6019F77DF91CF91FF9025
:105EA000EF90DF90CF90BF90AF909F908F9008952C
:105EB0000E940C2F089586E091E00E940C2F089517
:105EC0006093060170930701809308019093090184
:105ED00008952F923F925F926F927F928F929F923E
:105EE000AF92BF92CF92DF92EF92FF920F931F93E8
:105EF000CF93DF938B01EA016115710521F0DB017E
:105F00008C9311969C93209739F09E012250310971
:105F10002332310508F0D8C07C016701BFEFCB1AEE
:105F2000DB0A5601F7016080862D90E00E949B30CD
:105F3000892B11F07601F1CFFDE26F120AC05701F3
:105F400082E0A80EB11CD70111966C90772473944F
:105F50000BC0BBE26B1207C05701E2E0AE0EB11CF2
:105F6000D70111966C90712CCE018F7E892B89F40C
:105F7000B0E36B1237C0F50180818F7D8835D1F495
:105F80006180F2E0AF0EB11C872D8260782EC0E1F7
:105F9000D0E0CA30D10551F1C031D10521F0C8306F
:105FA000D10599F409C0CC24CA94DC2CEC2CAFE0C8
:105FB000FA2E22C0209769F7C8E0D0E0CC24CA941A
:105FC000DC2CEC2CFFE1FF2E17C06FEF7FEFCB0135
:105FD0009E01442737FD4095542F0E947A2E690177
:105FE0007A010AC02097A9F6CAE0D0E0E9E9CE2EEE
:105FF000DC2CEC2CE9E1FE2EF50160E020E030E045
:10600000A9014E01AA2497FCA094BA2C1F0170ED9F
:10601000572E560CA9E0A51570F48FEB860D8A312A
:1060200018F499EC592E06C08FE9860D8A3148F58F
:1060300089EA582E560C852D90E08C179D070CF59B
:106040006F3FD9F0C216D306E406F50698F0C501F5
:10605000B4010E94562E9B01AC01852D90E0A0E07A
:10606000B0E0280F391F4A1F5B1F281739074A075E
:106070005B0710F46FEF01C061E03196D1016C90C5
:10608000C5CF0115110551F0662311F0319703C0FA
:1060900071FE04C03297D801ED93FC9370FE07C0E7
:1060A00050954095309521953F4F4F4F5F4F67FF7B
:1060B00010C082E290E090938D0680938C066FEF83
:1060C0007FEF8FEF9FEF07C060E070E080E090E02F
:1060D00002C0B901CA01DF91CF911F910F91FF90CA
:1060E000EF90DF90CF90BF90AF909F908F907F9078
:1060F0006F905F903F902F900895FC01882799271B
:10610000E89421912032E9F3293010F02E30C8F3C1
:106110002B3241F02D3239F4689404C00E94CF3004
:10612000820F911D219120532A30C0F31EF49095C7
:1061300081959F4F0895911150C0803219F0895078
:106140008550D0F7089548EC53E00E94A830089598
:10615000FA01A191B081009719F41097E1F0CD01F7
:10616000DC01CD010D90002011F4C00113C0FB0132
:106170002191222319F02015D9F7F3CFFB012191AA
:10618000201519F41E92119606C02223C1F70D9016
:106190000020A1F7D001FA01A193B08308957AE01D
:1061A000979F902D879F802D910D11240895F99927
:1061B000FECF92BD81BDF89A992780B50895262F0C
:1061C000F999FECF1FBA92BD81BD20BD0FB6F894DC
:1061D000FA9AF99A0FBE019608959927882708958B
:0461E000F894FFCF61
:1061E40000008E06200001000000FF0002000200F3
:1061F400020002000200020002000200020002008B
:1062040002000200020002000200028025000005D4
:10621400400AA1204EA50020244EA52C2330C012F4
:1062240000001A400AA1204EA5001B1E27522C2351
:10623400308025000005400AA1204EA50020244EF0
:10624400A52C2330004B000006400AD0009D4900D5
:106254007B289D492C233000E1000005400A4501BC
:10626400D7DC03B81E0EBF00232E48E801008A4085
:106274000A6001555502AD1E20000023C801545880
:106284002074696D656F75742100596573004E6FD4
:10629400002C00386368004E2F41002C205B005D09
:1062A4002028002900486F70206368616E6E656C59
:1062B400200020402000456E746572696E6720617D
:1062C40064617074697665206368616E6E656C20C4
:1062D40073656C656374696F6E2C207069636B6998
:1062E4006E673A007363616E6E6572206D6F6465EC
:1062F400004E4F5420454E41424C45440053656E78
:1063040064696E672073657474696E677320746F53
:106314002052580A00526573657474696E6720735D
:10632400657474696E6773206F6E2052580A004159
:10633400626F727465642065646974730A00696EBF
:1063440076616C69642073656C656374696F6E0053
:106354000D0A496E76616C696420696E70757420EB
:106364002D20646973636172646564210700536559
:106374007474696E677320736176656420746F202A
:10638400454550524F4D0A005265766572746564F6
:106394002073657474696E67732066726F6D20452F
:1063A4004550524F4D0A004C6F616465642066612C
:1063B40063746F72792064656661756C74730A0026
:1063C4004B657920616E64206368616E6E656C73E1
:1063D4002072616E646F6D697A65640A004F70653E
:1063E4006E4C52536E6720545820737461727469F2
:1063F4006E672000206F6E20485720006D6F647513
:106404006C65206C6F636B65643F00342B3400381B
:1064140000382B340031320031322B340031360055
:1064240050504D0052535349005344410053434C80
:1064340000525844005458440041494E004C4245CF
:1064440045500053504B54524D0053425553005342
:10645400554D44004C4C494E440000070B0C1011A0
:106464001500B7012B032F033103350338033D0314
:10647400B7014003440349034D0351035503590332
:106484005D0363036A036F0374038D028D028D023F
:106494008D02160A13223129000000007C2C812A67
:0864A400222C4F2C342C712C2A
:107E00000F92CDB7DEB7112484B714BE81FFF1D035
:107E100082E08093C00088E18093C10086E0809377
:107E2000C20080E18093C4008EE0CDD088249924E4
:107E3000CC24C394F5E0DF2EE1E1EE2E73E0F72EC3
:107E4000B6D0082F813479F4B2D08983C2D0898129
:107E5000823811F481E005C0813811F485E001C059
:107E600083E09ED09AC0823411F484E103C085344B
:107E700019F485E0B6D091C0853561F498D0082F0B
:107E800010E095D090E0982E8824802A912A880CC2
:107E9000991C82C0863521F484E0A3D080E0E1CF34
:107EA000843609F04CC083D082D0A82E80D0B82E62
:107EB00000E011E07CD0F80181938F01AE16D1F77C
:107EC00088D0FB2DF53489F4E0E0F1E00BC0F9999E
:107ED000FECF92BC81BC0894811C911C819180BD15
:107EE000FA9AF99AEA1598F358C08B2D863409F05E
:107EF00054C0F401F7BEE89507B600FCFDCFF401CD
:107F0000A0E0B1E02C9130E011968C91119790E0B7
:107F1000982F8827822B932B12960C01C7BEE895C9
:107F20001124329681E0A038B80761F7F401D7BE7A
:107F3000E89507B600FCFDCFE7BEE8952EC0843774
:107F4000F1F435D034D0182F32D0B82E42D0FB2DDA
:107F5000F63421F4F40105914F010CC0FB2DF534EA
:107F600049F4F999FECF92BC81BC0894811C911C04
:107F7000F89A00B5802F14D0115049F70EC08537FC
:107F800039F427D08EE10CD085E90AD08FE069CF93
:107F9000813511F488E017D01CD080E101D050CF9A
:107FA0009091C00095FFFCCF8093C600089580910A
:107FB000C00087FFFCCF8091C00084FD01C0A89560
:107FC0008091C6000895E0E6F0E098E19083808318
:107FD0000895EDDF803219F088E0F5DFFFCF84E10E
:107FE000DFCF1F93182FE3DF1150E9F7F2DF1F9166
:0E7FF0000895282E80E0E7DFEE27FF27099492
:027FFE0001057B
:0400000300007E007B
:00000001FF
